:107446000000050200000301FA0400EF0500030A2C
:107456000A5A0B001E0C00FA0D00030E00040F0161
:1074660064100096120132130AFA14010217010A77
:107476001801EF1905321A010A1B01EF1C05321F0C
:10748600FFFF20FFFF23011E2400642A00FA2B00C1
:10749600FA2C50782D003D2E00463000643250788C
:1074A6003300003432FF3501643601643701503849
:1074B6000A643A00033B00043C00643E003C3F0083
:1074C6000140FFFF411450420A5A430AC84405329C
:1074D6004500B44600FA4900024B00014C00FA5040
:1074E6000606510596520A32530B46540A9657051C
:1074F60046590A465A32FA5B010A5C0A325E000AAB
:107506005F00646200FE64021C67FFFF6801016998
:1075160001016A05966B00006C32FF6D0004730072
:10752600017400017801327901327E0064810064C1
:1075360084FFFF8800028A00019D0A969E00019F33
:10754600FFFFA0013CA2000AA3FFFFA40064A50060
:1075560064A6FFFFA7FFFFA8FFFFA9FFFF010178B1
:107566001500022F003C4701784802045601044EDC
:10757600FFFF58000261FFFF6600028500AF86002C
:10758600018700FA890109990006A100FAFAFAFAB8
:1075960001013C1500022F1E3C47017848020456A3
:1075A60001034EFFFF58000261FFFF6600028500DF
:1075B600AF8600018700FA890109990000A1000041
:1075C600FAFAFA01013C1500002F1E3C47013C481F
:1075D60002035601014EFFFF58000061FFFF6600DF
:1075E6000085FFFF86FFFF87FFFF890102990000E4
:1075F600A10000FAFAFA0065006F00790083008D99
:10760600009700A100AC00B600C000CA00D400DE9E
:1076160000E800F200580060006800700078008002
:1076260000880090009800A000A800B000B800C133
:1076360000C800D000D800DF00E600EE00F60041EA
:107646000047004D00530059005F0065006C007153
:107656000077007D00830089008F0095009B00A2C3
:1076660000A700AC00B200B900C000C500CA00D235
:0A76760000D500DD00E100E700EFA1
:103D750075A71085F97485FA757E017F00E57512C2
:103D85007792E5742FFF50010E8E5A8F5B900018C5
:103D9500E0FCA3E0FDEF2DFDEE3CFC8C5C8D5D9021
:103DA5000038E0FAA3E0FBED2BFBEC3AFA8A5C8BDA
:103DB5005D2275A71085F97485FA757E017F00E58A
:103DC50075127792E5742FFF50010E8E5A8F5BACFA
:103DD5002DAD2EEF2DFDEE3CFC8C5C8D5D900038FD
:103DE500E0FAA3E0FBED2BFBEC3AFA8A5C8B5D2253
:103DF500E55DF5FBE55CF5FCD29322E55DF5E9E5CE
:103E05005CF5EAD29422E55DF5EBE55CF5ECD29143
:103E150022E55DF5EDE55CF5EED29222E55DF5FD79
:103E2500E55CF5FED28722E55DF5CEE55CF5CFD202
:103E35009022A203B34008E5B54480F5B58006E5B8
:103E4500B5547FF5B522E50C906FD8F82828730294
:103E55003EE7A23CB34008E5B54408F5B58006E564
:103E6500B554F7F5B5807BA23CB34008E5B54402EF
:103E7500F5B58006E5B554FDF5B58066A23CB340C1
:103E850008E5B54410F5B58006E5B554EFF5B58000
:103E950051A23CB34008E5B54420F5B58006E5B52B
:103EA50054DFF5B5803CA23CB34008E5B54440F588
:103EB500B58006E5B554BFF5B58027A23CB34008EB
:103EC500E5B54480F5B58006E5B5547FF5B58012B6
:103ED500A23C9292800CA23C92878006A23C9290D2
:023EE50080005B
:106FD800023E54023E57023E6C023E81023E960239
:106FE8003EAB023EC0023ED5023EDB023EE1023E1F
:016FF800E7B1
:103EE70022743690015FF07430900160F0742D9069
:103EF7000161F07432900162F07420900163F074F4
:103F070036900164F07443900165F074799001660E
:103F1700F0746C900167F07420900168F074209041
:103F27000169F0742090016AF0742090016BF074BD
:103F37002090016CF0742090016DF022900896E0BB
:103F4700FEA3E0FF741DD39F74019E400C9074463E
:103F5700120048E493F599804C90F802E493B40575
:103F670014900896E0FEA3E0FF907479120048E4ED
:103F770093F599803090F802E493D3940540149018
:103F87000896E0FEA3E0FF907446120048E493F51C
:103F9700998012900896E0FEA3E0FF9074AC12009F
:103FA70048E493F5999008961277A0900896E0FE5A
:103FB700A3E0FFEFB45007EEB40103754E0022AE45
:103FC7005AAF5B74068E048F05FF1277828C5C8D67
:103FD7005DAE5AAF5B74068E048F05FF1277AD8C0A
:103FE7005A8D5BC200E55B455A60137406C3955B47
:103FF700FFE4955AFE8E5A8F5B785C1277E5E5747D
:10400700A85CB80015D3955D4010E574C3955DFFB6
:10401700E4955CFE8E5C8F5D8012E574243CC3954D
:104027005DFFE4955CFE8E5C8F5DD200AE5CAF5D9C
:10403700743B6F4E6006743C6F4E701AAE5CAF5D9A
:10404700743B6F4E70057574018003757402755D5E
:104057003A755C0080037574002290009CE0B401FF
:1040670004C2078002D20790009DE0B40104C20891
:104077008002D2089000DAE075F0D2A4FFAEF074A7
:104087000A8E048F05FF12778290088AECF0A3ED61
:10409700F09000DAE075F02BA4FFAEF0900014EE7C
:1040A700F0A3EFF07E017F00900098E012779290E6
:1040B70000DBE08E048F05FF127782740AFF127708
:1040C700828D619000E4E075F0D2A4FFAEF0740A2F
:1040D7008E048F05FF12778290088EECF0A3EDF027
:1040E7009000E6E060139000E6E0F5F0741684FFB8
:1040F7007E00EF9008ECF0800674649008ECF09076
:1041070000DCE0900076F0900128E0900083F090CA
:10411700012AE0FE9000D8E08E0088F0A4FFAEF000
:10412700EF9008F5F0900103E075F013A4FDACF0F3
:10413700900038ECF0A3EDF0A225B340169001747F
:10414700E0700C900175E07006900176E0600280E7
:1041570002C225900174E0B4300F900175E0B447B6
:1041670008900176E0643B60028004D2268002C298
:1041770026900095E0FE9008F6E06E601B7599E6C4
:1041870012019C74AB900050F01206DA7464F509C2
:1041970075080012062480FE90008DE070067400FA
:1041A7009000C2F090007AE0FE9000C2E0B506638E
:1041B70090007DE0FE9000E0E0B5065790007BE0C0
:1041C700FE9000EEE0B5064B900081E0FE90009572
:1041D700E0B5063F90007EE0FE9000D0E0B50633E4
:1041E70090007CE0FE9000DEE0B5062790007FE0BF
:1041F700FE9000FBE0B5061B900080E0FE9000FCFF
:10420700E0B5060F900082E0FE90010EE06E7003AD
:104217000244C290009DE070089000DEE0640460F4
:1042270002800674039000DEF0900058E0C3940506
:1042370050087402900111F0801D9000D0E0D394D3
:104247000250069000EEE060087406900111F080BD
:10425700067409900111F0900095E0B4010674000E
:10426700900095F0900095E0B4020674009000E08D
:10427700F0900095E0B4030674009000EDF0900014
:10428700E0E0D394014026741B900113F074009072
:1042970000A9F074009006DEF074009006DFF0903D
:1042A70000C2E0600674009000C2F080329000C245
:1042B700E0601A7400900113F0741B9000A9F07469
:1042C700009006DEF074009006DFF0801274009014
:1042D7000113F074009000A9F0741B9006DEF090B3
:1042E70000D0E0D3940240089000EEE06402600240
:1042F700800674009000EEF09000D0E0D394024066
:10430700089000EEE0640160028027741C9001149D
:10431700F074009000AAF074009006E2F074009028
:1043270006E3F09000C2E0B4020674019000C2F008
:1043370080339000C2E0B4021A7400900114F07444
:104347001C9000AAF074009006E2F074009006E357
:10435700F080127400900114F074009000AAF074B9
:104367001C9006E2F09000FBE060147407900115C2
:10437700F074009006D6F074009006D7F0800C74A5
:1043870000900115F074079006D6F09000FCE060ED
:10439700147408900116F074009006DAF074009017
:1043A70006DBF0800C7400900116F074089006DAB2
:1043B700F090010EE06014742A900786F074009064
:1043C70006D2F074009006D3F0800C740090078634
:1043D700F0742A9006D2F09000D0E0B40206900064
:1043E700EEE06002802674049006E6F074059006FD
:1043F700EAF074069006EEF07400900781F07400FE
:10440700900782F07400900783F08036740090065E
:10441700E6F074009006E7F074009006EAF0740086
:104427009006EBF074009006EEF074009006EFF043
:104437007404900781F07405900782F07406900762
:1044470083F09000DEE0D39402401474189007794B
:10445700F0741990077AF0741A90077BF080127441
:1044670000900779F0740090077AF0740090077B4A
:10447700F0D2249000C2E090007AF09000EEE09035
:10448700007BF09000E0E090007DF09000D0E0909D
:10449700007EF09000DEE090007CF0900095E090C8
:1044A7000081F09000FBE090007FF09000FCE0902E
:1044B7000080F090010EE0900082F09000F8E0B4E8
:1044C7000117900024740FF0A374FFF0900026E406
:1044D700F0A3F074029000F8F09000F8E0B4034104
:1044E700900026E0FEA3E0FF900024E0FCA3E0FD9F
:1044F7001277DD74101277927408120039EF90006A
:10450700F7F0EF700674FF9000F7F074009000F872
:10451700F0900025E09000AEF0900024E09000AF0E
:10452700F0900089E0900086F0900088E090008588
:10453700F09000B7E0C3941E50569000B7E0F40423
:10454700241E900087F0900087E075F00684FF7EB8
:10455700008F74900087E075F00684ADF07C008DC5
:1045670075900085E0D39575400D900085E0C39563
:1045770075900085F0800F900085E02406C395753F
:10458700900085F00574900086E02574900086F011
:10459700900086E0900046F0900046E024149000DA
:1045A70047F0900046E02428900048F0900046E04D
:1045B700D39478400B900046E0C39478900046F07F
:1045C700900047E0D39478400B900047E0C394787D
:1045D700900047F0900048E0D39478400B90004853
:1045E700E0C39478900048F0C228900046E0D39446
:1045F7003C400D900046E0C3943C900046F0D22822
:10460700C229900047E0D3943C400D900047E0C397
:10461700943C900047F0D229C22A900048E0D394F6
:104627003C400D900048E0C3943C900048F0D22AEB
:1046370090004CE4F0900046E0643B600790004631
:10464700E0B43C20900046E0B43B06740290004C76
:10465700F0900046E0B43C0690004C7401F09000E6
:10466700467401F090004DE4F0900047E0643B6031
:1046770007900047E0B43C20900047E0B43B067445
:104687000290004DF0900047E0B43C0690004D7456
:1046970001F09000477401F090004EE4F09000485C
:1046A700E0643B6007900048E0B43C20900048E09D
:1046B700B43B06740290004EF0900048E0B43C060C
:1046C70090004E7401F09000487401F0900089E06A
:1046D700FE9000ECE02E900051F0900051E0D39452
:1046E7003C400B900051E0C3943C900051F0900087
:1046F70051E0D3943C400B900051E0C3943C9000B0
:1047070051F09000C7E0B40163900051E0641E606F
:1047170007900051E0B43C06900051E004F090008F
:1047270051E0641D6007900051E0B43B06900051D2
:10473700E014F0900051E0D3943C400B900051E01E
:10474700C3943C900051F0900051E0D3941E400D6B
:10475700900051E0C3941E900052F0800A900051DF
:10476700E0241E900052F0755E1E8079900051E0A3
:104777006414600F900051E064286007900051E0D6
:10478700B43C06900051E004F0900051E0641360DF
:104797000F900051E064276007900051E0B43B069A
:1047A700900051E014F0900051E0D3943C400B90FE
:1047B7000051E0C3943C900051F0900051E0D39435
:1047C70014400B900051E0C39414900051F09000F6
:1047D70051E0D39414400B900051E0C3941490001F
:1047E70051F0755E14900089E0FE9000CFE0D39EF3
:1047F7005013900089E0FE9000CFE0F4042E04905F
:104807000049F08013900089E02478FE9000CFE003
:10481700F4042E04900049F0900049E075F01484E8
:10482700AFF07E00EF4E7006900049E004F0900074
:1048370049E00475F01484AFF07E00EF4E700690E7
:104847000049E014F0900049E0B4790690004974FB
:1048570001F0900049E0D3943C400F900049E0C339
:10486700943C900049F0D21F8002C21F900049E09B
:10487700241490004AF0900049E0242890004BF05F
:1048870090004AE0D3943C400B90004AE0C3943C2C
:1048970090004AF090004BE0D3943C400B90004BC3
:1048A700E0C3943C90004BF012019C22C293C29447
:1048B700C291C292C287C290E5B554EFF5B5E5B58E
:1048C70054DFF5B5C296C295C2A0C297C2A2C2A1D3
:1048D700E5B554BFF5B5E5B5547FF5B5E5B554FB7A
:1048E700F5B5C209755F469000D2E07005756E0296
:1048F7008003756E0375550075540090000C74FFA6
:10490700F0A374DCF0C20FC212C21574C890003A4B
:10491700F074C890003EF074C8900042F0755300E0
:10492700755200C204754700E570B4130375700033
:1049370075640090001AE4F0A3F0757110C20CC200
:104947000DC20EC20375570075560090000EE4F0B5
:10495700A3F0900010E4F0A3F0C22C75590075582D
:1049670000900094E075F032A4FFAEF0900022EEC4
:10497700F0A3EFF0900084E4F09008F2E4F0C2278F
:10498700D21CC21BD21DC21EC21FC220900012E43D
:10499700F0A3F022755B00755A00AE5AAF5B741C2A
:1049A700C39F74019E5003024A8F907446120048B9
:1049B700E493645F6023907446120048E493647E36
:1049C7006017907446120048E4936481600B9074FA
:1049D70046120048E493B48403024A6FAE5AAF5BB1
:1049E700907446120048E4939000881277C30FBF73
:1049F70000010EE0FC907446120048ECFEE493FFC1
:104A0700EEC39F5026AE5AAF5B0FBF00010E9074E6
:104A170046120048AE5AAF5BE493FC90744612000E
:104A270048E4939000881277C3ECF0AE5AAF5B90DE
:104A37007446120048E4939000881277C3E0FC9014
:104A47007448120048ECFCE493FDECD39D401990A8
:104A57007448120048E493FC907446120048E493AB
:104A67009000881277C3ECF0AE5AAF5B74022FFF49
:104A770050010E8E5A8F5B785B740126F65004182E
:104A8700E436F640030249A122755B00755A00AE71
:104A97005AAF5B7432BE00039F5003024B5D9075A3
:104AA70063120048E4939000881277C30FBF000198
:104AB7000EE0FC907563120048ECFEE493FFEEC332
:104AC7009F5026AE5AAF5B0FBF00010E9075631261
:104AD7000048AE5AAF5BE493FC907563120048E45C
:104AE700939000881277C3ECF0AE5AAF5B90756372
:104AF700120048E4939000881277C3E0FC90756534
:104B0700120048ECFCE493FDECD39D4019907565C9
:104B1700120048E493FC907563120048E4939000F8
:104B2700881277C3ECF0AE5AAF5B742D6F4E7006E8
:104B3700755B33755A00AE5AAF5B74022FFF500195
:104B47000E8E5A8F5B785B740126F6500418E43694
:104B5700F64003024A9622755B00755A00AE5AAFBB
:104B67005B7432BE00039F5003024C2B9075961264
:104B77000048E4939000881277C30FBF00010EE04E
:104B8700FC907596120048ECFEE493FFEEC39F502D
:104B970026AE5AAF5B0FBF00010E90759612004804
:104BA700AE5AAF5BE493FC907596120048E493907D
:104BB70000881277C3ECF0AE5AAF5B90759612007F
:104BC70048E4939000881277C3E0FC907598120030
:104BD70048ECFCE493FDECD39D40199075981200C6
:104BE70048E493FC907596120048E493900088126D
:104BF70077C3ECF0AE5AAF5B742D6F4E7006755BE2
:104C070033755A00AE5AAF5B74022FFF50010E8EF8
:104C17005A8F5B785B740126F6500418E436F64029
:104C270003024B6422755B00755A00AE5AAF5B7482
:104C370032BE00039F5003024CF99075C912004819
:104C4700E4939000881277C30FBF00010EE0FC9039
:104C570075C9120048ECFEE493FFEEC39F5026AEE1
:104C67005AAF5B0FBF00010E9075C9120048AE5ACC
:104C7700AF5BE493FC9075C9120048E493900088F9
:104C87001277C3ECF0AE5AAF5B9075C9120048E4D7
:104C9700939000881277C3E0FC9075CB120048EC24
:104CA700FCE493FDECD39D40199075CB120048E4CA
:104CB70093FC9075C9120048E4939000881277C35B
:104CC700ECF0AE5AAF5B742D6F4E7006755B3375A3
:104CD7005A00AE5AAF5B74022FFF50010E8E5A8FE7
:104CE7005B785B740126F6500418E436F64003023D
:104CF7004C322275A71085F97485FA757E017F00FD
:104D0700E575127792E5742FFF50010E8E5A8F5B6F
:104D1700AC5CAD5DEF2DFDEE3CFC8C5C8D5D123D1A
:104D2700F5123E00123E0B9000D0E0D394024009EA
:104D3700123E16123E21123E2C75A7002285F974E9
:104D470085FA757E017F00E575127792E5742FFF6E
:104D570050010E8E5A8F5B7E017F7690010DE01217
:104D67007792AC5AAD5BED2FFFEC3EFE8E5C8F5D0C
:104D7700E55DF5EDE55CF5EE900076E4F0741290F4
:104D87000054F02285F97485FA757E017F00E57578
:104D9700127792E5742FFF50010E8E5A8F5B9000A9
:104DA70014E0FCA3E0FDEF2DFDEE3CFC8C5C8D5D7B
:104DB700E55DF5FDE55CF5FE22056522A2DBB34066
:104DC700089000DCE0900076F0A2DCB34048A296A1
:104DD70050067419900054F0A2955006741990006B
:104DE70054F0A2A050067419900054F0A2975006F0
:104DF7007419900054F0A2A250067419900054F050
:104E0700A2A150067419900054F0C296C295C2A090
:104E1700C297C2A2C2A175D8402285A77375A710F1
:104E27009000D0E0D3940250079000EEE0B4025215
:104E3700A2D8B34002C293A2D9B34002C294A2DA65
:104E4700B34002C2919000D0E0640260079000D0A6
:104E5700E0B40417A2DBB34002C292A2DCB3400263
:104E6700C287A2DDB34002C2908015A2D8B3400228
:104E7700C292A2D9B34002C287A2DAB34002C2905B
:104E8700802DA2D8B3400AC2939000EEE06002C220
:104E970092A2D9B3400AC2949000EEE06002C287A2
:104EA700A2DAB3400AC2919000EEE06002C29075A8
:104EB700D8408573A72290F800E4936406600280C7
:104EC700FE12009E75A70075D80075D90475DD0917
:104ED70075DE0975D84075A71075D80075D90475A2
:104EE700DA0975DB0975DC0975DD0975DE0975DF1A
:104EF7000975D84075A7001200FB74C8F509750835
:104F07000012062475A70FE5FC900063F0E5FB90FF
:104F17000064F0E5FA900065F0E5F9900066F07539
:104F2700A70090F800E493F52812074390089FE044
:104F3700D39403500790089FE0B4010674009008CB
:104F47009FF090089FE09008F6F074019000D1F070
:104F570090089FE0906FF9F8282873802A802875B9
:104F6700A70F75F30F75A700A2A340067402900060
:104F7700D1F0801375A70F75F31775A700A2A4408A
:074F87000674029000D1F056
:0C6FF900024F62024F64024F66024F7BA1
:104F8E009000D1E0B4022AC21A120AEC7402900008
:104F9E00D1F090089FE0907005F82828738010805B
:0F4FAE000E74009000E0F0800674009000EDF0AB
:0C700500024FAB024FAD024FAF024FB77D
:104FBD008028D21A120A0174019000D1F090089F36
:104FCD00E0907011F82828738010800E7400900006
:0A4FDD00E0F0800674009000EDF093
:0C701100024FD5024FD7024FD9024FE1C9
:104FE70090F807E493900070F0900070E044089008
:104FF7000070F0900070E054FE900070F01203BD56
:10500700123EE89008ACE0900174F09008ADE09093
:105017000175F09008AEE0900176F0900174E070B1
:105027000C900175E07006900176E060028004C282
:10503700258002D2259000C2E00490007AF090010A
:105047002CE0B4FF06740090012CF090012DE0B421
:10505700FF06740090012DF012499B90F802E4932B
:10506700B40505124B5E801290F802E493D39405C1
:105077004005124A908003124C2C74009000F8F0FF
:10508700124061E5B54401F5B57406900056F07419
:1050970000900057F07401900058F090F802E493E4
:1050A700900059F090F803E49390005AF090F804B8
:1050B700E49390005BF0740690005CF0900059E078
:1050C700B40506740590005CF0900059E0B404063E
:1050D700740490005CF0741E90005DF074039000FF
:1050E7005EF0740790005FF07401900060F090F834
:1050F70005E493900061F090F806E493900062F065
:10510700740090006AF0740090006BF074009000D7
:105117006CF0740090006DF0740090006EF07400F5
:1051270090006FF074FF900071F0A2B6B39205A2E1
:10513700B3B39206A2A4B39222A2A3B39223900080
:1051470072E4F0757000743A900788F074FD900768
:1051570089F0900073E4F0756F01900054E4F090CB
:1051670000D2E0B40106741A900054F0C2217564AD
:1051770000C20AD20BC203757200C2241205C6759B
:105187006000756C0075620075663275670075683A
:1051970000756900756A00756B0090001AE4F0A34A
:1051A700F0756D00D2B2D2A4D2B0D2B1D2A3D2A739
:1051B700D2A6D2A5D2B77E017F009000AFE01277CA
:1051C700929000AEE02FFF50010E900024EEF0A366
:1051D700EFF0EFD394FFEE940F4007900024E4F034
:1051E700A3F09000F7E0700674FF9000F7F09000CE
:1051F700D2E07005756E028003756E03740090012E
:1052070017F07400900118F074299006CEF0741509
:10521700900776F07416900777F07417900778F078
:10522700740090077CF0740090077DF0740190077C
:105237007EF0740290077FF07403900780F074008B
:10524700900784F07400900785F0D29CE571D394A1
:105257001040037571109006CFE0D3940C4006748C
:10526700009006CFF09006D3E0D3940C400674006C
:105277009006D3F09006D7E0D3940C4006740090C4
:1052870006D7F09006DBE0D3940C40067400900636
:10529700DBF09006DFE0D3940C400674009006DF45
:1052A700F09006E3E0D3940C400674009006E3F018
:1052B7009006E7E0D3940C400674009006E7F09060
:1052C70006EBE0D3940C400674009006EBF09006D2
:1052D700EFE0D3940C400674009006EFF0D2EC7523
:1052E700CF01A298B34005C298120C54E54E600650
:1052F700A299B3B340028005C2991210E0E54F644A
:10530700016005E54FB4040280D5C28E7E107F0090
:10531700E565127792E58D75F010A4FDACF0EF2DE1
:10532700FDEE3CFCE58B75F01084FF7E00ED2FFF52
:10533700EC3EFE8E548F55D28E9000B5E0600990FA
:1053470000B5E0C3943D4002805690001C1277A040
:1053570090001CE0FEA3E0FF90001EE0FCA3E0FD30
:10536700EFB5053CEEB50438B218A204B34013A25A
:1053770018B34008E5B54404F5B58006E5B554FB18
:10538700F5B590001EE0FEA3E0FF900020E0FCA32F
:10539700E0FDEF2DFDEE3CFC90001EECF0A3EDF0E0
:1053A7009000C2E060099000C2E0C394034003028A
:1053B700545E123027A20440089000ACE0F5468006
:1053C7001BE560C395615005754600800F900099F5
:1053D700E0C3956250069000BFE0F546E54675F0DC
:1053E70002A4FFAEF0900894EEF0A3EFF0AC2FAD5F
:1053F70030EDD39FEC9E402CE5B554BFF5B5900634
:10540700CFE07006E5B554F7F5B59000C2E0B402F9
:10541700099000E0E0C3940240028006E5B54480AD
:10542700F5B58033900072E0C39441502AE5B54446
:1054370040F5B59006CFE07006E5B54408F5B590A0
:1054470000C2E0B402099000E0E0C3940240028089
:1054570006E5B5547FF5B59000C2E0B403241231D8
:1054670042AE2FAF30900894E0FCA3E0FDEFD39D50
:10547700EE9C4008E5B54440F5B58006E5B554BF58
:10548700F5B590009DE06009A2B3300601B3B340C3
:10549700028056A2B3300601B3404EA2B3300801D2
:1054A700B34039A21C4030900083E0D3955F40257C
:1054B7009008F2E07013900084E0B401069008F2BF
:1054C7007401F0900084E004F0A21BB34005900043
:1054D70084E4F0D21BD21CA208B39206A208B33010
:1054E700B301B34004A2089206A2B6300501B35037
:1054F70003025C28A2B6300501B35003025C28A260
:10550700B6300701B35003025B46756F009000B5D4
:10551700E0B43D13A207B34008E5B554FBF5B580E9
:1055270006E5B54404F5B5055FA209B3B35013AE5C
:1055370054AF5590000CE0FCA3E0FDEDC39FEC9E3B
:105547004003025711E56EB4032EA22CB34022E5A7
:105557005FB43B03756E01E55FC3943B5006900053
:10556700547401F0E55FD3943B40067402900054F5
:10557700F0755F01D22C8066E56EB4020A756E0184
:10558700755F3BC21BC21DE55FB43B05755F0180BC
:105597004D900054E07038E55FC3943B500690008F
:1055A700547401F0E55FD3943B40067402900054B5
:1055B700F0E55FC3943B5002D221E55FD3943B40B3
:1055C70002D221C296C295C2A0C297C2A2C2A1901E
:1055D70000D2E0B401051248B38003755F01AE56EF
:1055E700AF57AC54AD55EF2DFDEE3CFC74028C0665
:1055F7008D071200398E568F579000B5E0600990DD
:1056070000B5E0C3943D4002804390001CE0FEA338
:10561700E0FF9000B5E08E048F05FF1277827401DA
:105627008C068D07120039900020EEF0A3EFF09062
:105637000020E0F8A3E090001EC8F0A3C8F0900097
:105647001CE4F0A3F0C218E5B554FBF5B5A2A4B36A
:105657004002C222A2A3B34002C223A221B3400246
:10566700C221B21E9008F2E0B40111A21BB340049C
:10567700D21E8002C21E74029008F2F09008F2E077
:10568700C394025006A204B3B3400280067402908A
:1056970008F2F09000DEE0640460079000D0E0B408
:1056A700046290009DE060069008F2E07002800DB1
:1056B700A21D301B01B34005900084E4F09000D296
:1056C700E064016006A227B3B3501790009DE06025
:1056D70009A21B301D01B3B3400280067405900078
:1056E70054F0B21DA21CB3401BA21BB34004D21D31
:1056F7008002C21D9000D2E070069008F2E07002AE
:105707008002D227C21BC21C803AAE56AF57AC5498
:10571700AD55EF2DFDEE3CFC74018C068D07120094
:10572700398E568F57E56EC39402500DAC54AD5564
:1057370074B8C39D740B9C400280091248B3740669
:10574700900054F0E55FB43B127403900054F0D21C
:10575700219000D2E0B401031248B3AE58AF59AC60
:1057670054AD55EF2DFDEE3CFC8C588D59AE54AF22
:1057770055EFD39DEE9C4011900012E0FAA3E0FB99
:10578700EBC394E8EA940340028006900012127774
:10579700A0900010E0FEA3E0FFAC54AD55EF2DFD47
:1057A700EE3CFC900010ECF0A3EDF09000D2E0B4DA
:1057B7000118AE54AF55740512779274011200396F
:1057C70090000CEEF0A3EFF08011AE54AF557402C9
:1057D70012779290000CEEF0A3EFF0C28E758D0059
:1057E700758B00756500755501755400D28EE55FA0
:1057F700240E75F00F84AFF07E00EF4E6003025861
:105807008AE56E6013AE56AF57740F127792900009
:105817000EEEF0A3EFF0800F900010E0F8A3E090F9
:10582700000EC8F0A3C8F090000EE0FEA3E0FFEF63
:105837004E600B7C797DC21276808E528F5390001A
:1058470010E4F0A3F0AE52AF537428BE00039F508C
:1058570010E5642FFF50010E74011200398E528F2C
:10586700538553649000D9E0A852B8000DD39553DF
:105877004008E553900053F080099000D9E0149058
:105887000053F09000D0E0B40408900049E0655F51
:105897006002800EA21E301F01B34004D220800296
:1058A700C220E55F640B6005E55FB429099000C27B
:1058B700E06003122CDD9000C7E0B40114900051A2
:1058C700E0655F6007900052E0B55F037570008088
:1058D7001E900051E0655F6013900051E02414654D
:1058E7005F6009900051E02428B55F03757000A23E
:1058F7000A5003025A699000DEE0C394045006A2DE
:1059070009B3B340030259B490008EE0B401739019
:105917000110E0B40214121281900077E075F0BC18
:10592700A4FFAEF08E5C8F5D8056E56875F00A8443
:10593700FF7E00900588120048E0F55B755A00AEBF
:105947005AAF5B9000B3E012779274648E048F05B0
:10595700FF1277828C5C8D5DE55D90004FF0AE5A4B
:10596700AF5B90008CE012779274648E048F05FF12
:1059770012778274BC8C068D071277928E5C8F5DCE
:10598700801790008CE075F0BCA4FFAEF08E5C8FA2
:105997005D9000B3E090004FF0E562C394CC5006F1
:1059A700E55D455C70028003124CFAD20A9000DE76
:1059B700E0B404069008F2E07003025A6990008E82
:1059C700E0B40173900110E0B40214121281900048
:1059D70077E075F0BCA4FFAEF08E5C8F5D8056E576
:1059E7006875F00A84FF7E00900588120048E0F58C
:1059F7005B755A00AE5AAF5B9000B3E012779274B2
:105A0700648E048F05FF1277828C5C8D5DE55D9057
:105A1700004FF0AE5AAF5B90008CE012779274643F
:105A27008E048F05FF12778274BC8C068D07127760
:105A3700928E5C8F5D801790008CE075F0BCA4FFA0
:105A4700AEF08E5C8F5D9000B3E090004FF0E562A2
:105A5700C394CC5006E55D455C70028003124CFA96
:105A6700D20AE56EB40106E55F6411600280189002
:105A770000DEE0B4040575710380097571009000BC
:105A8700557401F0756E00E56E6003025B4190008E
:105A9700D5E0600D900076E0A852B8000695534017
:105AA7000280409000D5E0B4021F900046E0655F99
:105AB700600F900047E0655F6007900048E0B55FC2
:105AC70003757103756D00800CC201756D00900040
:105AD7001AE4F0A3F0900076E06006740990005491
:105AE700F08057900046E0655F600F900047E065E3
:105AF7005F6007900048E0B55F409000DEE0B404C7
:105B07000FA227B3400575710080037571038003E9
:105B1700757100900046E0B55F069000557401F07E
:105B2700900047E0B55F067402900055F09000487A
:105B3700E0B55F067403900055F0A207B39205A283
:105B470007B330B601B35003025C28756F019000AC
:105B5700B5E0B43D13A207B34008E5B54404F5B575
:105B67008006E5B554FBF5B5E5B54401F5B5742BED
:105B7700900072F0A2079205E55FD3944A4014D2D1
:105B870009E55FD39485400B7405900054F0D2214A
:105B9700755F469000DDE0B40107E56BC3944140B3
:105BA700028018E56BC3941450087413900054F0E6
:105BB7008006740E900054F01248B390005CE0FE2B
:105BC700900059E0C39E4009900059E0D3940840E3
:105BD7000974FB900054F01248B390005AE0601526
:105BE70090005AE0FE900058E06E600974FC900047
:105BF70054F01248B390005BE0601590005BE0FE44
:105C070090005DE06E600974FE900054F01248B396
:105C170090089FE0600690010DE060028003120B80
:105C2700D7A221B3400CC296C295C2A0C297C2A206
:105C3700C2A190010DE0600CAE52AF537414BE00C8
:105C4700059F40028037900095E090701DF8282846
:105C570073802A8028A2A3B35005A223B3400280F1
:105C670005124D44D2238015A2A4B35005A222B336
:0D5C770040028005124D44D22280028000C0
:10701D00025C58025C5A025C5C025C6F025C82028C
:02702D005C8481
:105C8400A20CB3B35008900049E0655F6003025D65
:105C9400F2A202B35006A201B3B34003025DEC903A
:105CA40000D0E0B404028003025DB0123D75900898
:105CB400F2E0B402028003025D9EA220B34067902A
:105CC4000121E0601F900018E0FEA3E0FF9001199D
:105CD400E012779274C88E048F05FF1277828C5C71
:105CE4008D5D800A900018E0F55CA3E0F55DAE5C84
:105CF400AF5D745E12779274058E048F05FF127780
:105D040082AE5AAF5BED2FFFEC3EFE8E5C8F5D9052
:105D14000038E0FCA3E0FDEF2DFDEE3CFC8C5C8D37
:105D24005D123DF58068900121E0D39403401F90FB
:105D34000018E0FEA3E0FF90011CE012779274C803
:105D44008E048F05FF1277828C5C8D5D800A900033
:105D540018E0F55CA3E0F55DAE5CAF5D745E1277B0
:105D64009274058E048F05FF127782AE5AAF5BEDF5
:105D74002FFFEC3EFE8E5C8F5D900038E0FCA3E0CC
:105D8400FDEF2DFDEE3CFC8C5C8D5D123E1690000B
:105D9400EEE0B40103123E378010123DF5123E16B8
:105DA4009000EEE0B40103123E378039123D7512C3
:105DB4003DF59000D0E0B4030ED2929000EEE0B432
:105DC4000103123E37801E9000EEE0B40206123D3D
:105DD400B7123E169000EEE0B40106A203B3B3403E
:105DE400028002D29275A700C20CD20DD20EA20D6F
:105DF400B3B3500890004AE0655F6003025F73A28A
:105E040002B35006A201B3B34003025F6D9000D009
:105E1400E0B404028003025F21123D759008F2E0B1
:105E2400B402028003025F0FA220B3406A900121F2
:105E3400E0D39401401F900018E0FEA3E0FF90011E
:105E44001AE012779274C88E048F05FF1277828C41
:105E54005C8D5D800A900018E0F55CA3E0F55DAE12
:105E64005CAF5D745E12779274058E048F05FF1229
:105E74007782AE5AAF5BED2FFFEC3EFE8E5C8F5DFA
:105E8400900038E0FCA3E0FDEF2DFDEE3CFC8C5CC3
:105E94008D5D123E008068900121E0D39404401F80
:105EA400900018E0FEA3E0FF90011DE012779274C9
:105EB400C88E048F05FF1277828C5C8D5D800A90FA
:105EC4000018E0F55CA3E0F55DAE5CAF5D745E12B6
:105ED400779274058E048F05FF127782AE5AAF5BFA
:105EE400ED2FFFEC3EFE8E5C8F5D900038E0FCA34E
:105EF400E0FDEF2DFDEE3CFC8C5C8D5D123E2190AF
:105F040000EEE0B40103123E378010123E00123E50
:105F1400219000EEE0B40103123E378049123D7532
:105F2400123E009000EEE0C394025007A203B34077
:105F340002D2879000D0E0B4030ED2879000EEE046
:105F4400B40103123E37801E9000EEE0B402061244
:105F54003DB7123E219000EEE0B40106A203B3B3B4
:105F640040028002D28775A700D20CC20DD20EA2C5
:105F74000EB3B3500890004BE0655F60030260F419
:105F8400A202B35006A201B3B340030260EE900034
:105F9400D0E0B4040280030260A2123D759008F2BE
:105FA400E0B402028003026090A220B3406A900130
:105FB40021E0D39402401F900018E0FEA3E0FF907C
:105FC400011BE012779274C88E048F05FF1277824A
:105FD4008C5C8D5D800A900018E0F55CA3E0F55DB3
:105FE400AE5CAF5D745E12779274058E048F05FF0C
:105FF400127782AE5AAF5BED2FFFEC3EFE8E5C8FC4
:106004005D900038E0FCA3E0FDEF2DFDEE3CFC8C40
:106014005C8D5D123E0B8068900121E0D3940540B5
:106024001F900018E0FEA3E0FF90011EE01277929B
:1060340074C88E048F05FF1277828C5C8D5D800A94
:10604400900018E0F55CA3E0F55DAE5CAF5D745EB6
:1060540012779274058E048F05FF127782AE5AAFC1
:106064005BED2FFFEC3EFE8E5C8F5D900038E0FC14
:10607400A3E0FDEF2DFDEE3CFC8C5C8D5D123E2C0F
:106084009000EEE0B40103123E378010123E0B1272
:106094003E2C9000EEE0B40103123E378049123DDD
:1060A40075123E0B9000EEE0C394025007A203B3B6
:1060B4004002D2909000D0E0B4030ED2909000EE53
:1060C400E0B40103123E37801E9000EEE0B40206F5
:1060D400123DB7123E2C9000EEE0B40106A203B3C9
:1060E400B340028002D29075A700D20CD20DC20E2A
:0D60F400E57190702FF82828739000F5E0FA
:03702F000260FDFF
:106101009070BCF828287312260C801212260C807D
:0E6111000D12269680081227428003122742A4
:0F70BC0002610802610D02611202611702611C7C
:10611F0075710102664F12286E1229857571020280
:10612F00664F122D21A204B340139000DAE075F0F0
:10613F001DA4FFAEF0900014EEF0A3EFF0900888CE
:10614F00E0FEA3E0FF740A12779290000EE0FCA32A
:10615F00E0FD74098F02FF1277828D078C038E0486
:10616F008A058B0612768090088CEEF0A3EFF090E4
:10617F0000DEE0B401087450BE00059F4002800DA0
:10618F00745090088CF8E4F0E8A3F0801B90088C12
:10619F00E0FEA3E0FF74F0BE00039F500B74F0907D
:1061AF00088CF8E4F0E8A3F0E53770037537019039
:1061BF00088CE0FEA3E0FFE5372FFF50010E90089B
:1061CF008CEEF0A3EFF0757103A233401A900055D7
:0161DF00E0DF
:067032000261250261313C
:1061E0009070CBF8282873800D75710A800875713E
:0661F0000B800375710C29
:0C70CB000261E70261E90261EE0261F37C
:1061F60002664F9006CFE06006750801122E4FA288
:1062060035B3B35008900786E0642A60028009E53A
:10621600B54402F5B50262BF9000C3E0D3940240D4
:1062260045900097E02403A852B8000495535009FE
:10623600900099E0D395625002800ED202A22B40C4
:10624600067408900054F0D22B900097E0A852B83C
:106256000005D39553500B900099E02403C3956233
:106266005002C2028053900097E02403A852B8005F
:106276000495535010E560C395615009900099E06C
:10628600D395625002800ED202A22B40067408906B
:106296000054F0D22B900097E0A852B80005D39591
:1062A600535014E561240FC39560400B900099E0AC
:1062B6002403C395625002C202A2024002C22BA26C
:1062C60035B3500DA202B35008900786E0642A60E9
:1062D600028006E5B554FDF5B59000DDE07007E5F2
:1062E6006BC3941440028002D2029000D2E0B40143
:1062F60002D202A2024005757104800A75711090DF
:0D630600001AE4F0A3F002664F9000C3E01F
:067038000261F902630F82
:106313009070D7F82828731213978012121397805E
:0E6323000D12154A8008121601800312160191
:0F70D70002631A02631F02632402632902632EFD
:106331009006D3E06006750802122E4F75710502B2
:10634100664F12175A7571069006D7E060067508F8
:1063510003122E4F9006DBE06006750804122E4FE3
:1063610002664F90004FE06006A204B3B340028082
:106371000DE55FD39414500690004FE014F012190C
:10638100E37571079006DFE06006750805122E4F70
:106391009006E3E06006750806122E4F02664F90E4
:1063A1000110E0B40203121308121E4B757108901C
:1063B10006E7E06006750807122E4F9006EBE060D5
:1063C10006750808122E4F02664F121F2D757109AE
:1063D10002664F122305A20CB35005A20DB3400271
:1063E1008006D20CD20DD20E7571109006EFE060CE
:1063F10006750809122E4F02664F90003CE0C394C7
:1064010046500AC296C297744690003CF090004CE8
:10641100E0B4011DE5372406F53790088CE0FEA3B2
:10642100E0FF74062FFF50010E90088CEEF0A3EFF1
:10643100F090004CE0B4021DE537240CF5379008CC
:106441008CE0FEA3E0FF740C2FFF50010E90088C2E
:10645100EEF0A3EFF085375B755A00900046E0F54A
:1064610074123FC6E55D90003CF0900006E55AF0DD
:10647100A3E55BF0E57490003DF0C21090088CE05C
:10648100F55AA3E0F55B900046E0F574123FC6E5CE
:106491005D90003AF0900000E55AF0A3E55BF0E56D
:1064A1007490003BF0A200921190004CE06002B2A7
:1064B10011C20F75710302664F900040E0C394460C
:1064C10050139000DEE0B40102C296C295C2A274DC
:1064D10046900040F090004DE0B4011DE5372406E0
:1064E100F53790088CE0FEA3E0FF74062FFF500102
:1064F1000E90088CEEF0A3EFF090004DE0B4021D79
:10650100E537240CF53790088CE0FEA3E0FF740C0E
:106511002FFF50010E90088CEEF0A3EFF085375B52
:10652100755A00900047E0F574123FC6E55D900092
:1065310040F0900008E55AF0A3E55BF0E5749000A7
:1065410041F0C21390088CE0F55AA3E0F55B90008E
:1065510047E0F574123FC6E55D90003EF090000201
:10656100E55AF0A3E55BF0E57490003FF0A20092DC
:106571001490004DE06002B214C2127571030266FC
:106581004F900044E0C3944650139000DEE0B40104
:1065910002C296C2A0C2A17446900044F090004E7F
:1065A100E0B4011DE5372406F53790088CE0FEA321
:1065B100E0FF74062FFF50010E90088CEEF0A3EF60
:1065C100F090004EE0B4021DE537240CF537900839
:1065D1008CE0FEA3E0FF740C2FFF50010E90088C9D
:1065E100EEF0A3EFF085375B755A00900048E0F5B7
:1065F10074123FC6E55D900044F090000AE55AF040
:10660100A3E55BF0E574900045F0C21690088CE0BC
:10661100F55AA3E0F55B900048E0F574123FC6E53A
:106621005D900042F0900004E55AF0A3E55BF0E5CF
:1066310074900043F0A200921790004EE06002B205
:0E66410017C215757103800680048002800068
:10703E000263430263640263A00263CB0263D40261
:10704E0063FB0264BA02658202664902664B0266FF
:04705E004D02664F2A
:10664F0090003AE0B55F02800302672CA20F407200
:10665F00900000E0FEA3E0FFEF4E6021AE56AF5773
:10666F00900000E0FCA3E0FD12000374068E048F7F
:10667F0005FF127782900000ECF0A3EDF090003B45
:10668F00E0601A900000E0FEA3E0FFAC56AD57EFBC
:10669F002DFDEE3CFC900000ECF0A3EDF090003BE4
:1066AF00E0D39401401A900000E0FEA3E0FFAC5647
:1066BF00AD57EF2DFDEE3CFC900000ECF0A3EDF09C
:1066CF00D20FAE54AF55900000E0FCA3E0FDEFC336
:1066DF009DEE9C4048124D8B9000DEE0907062F86A
:1066EF002828738030D296802CD2968028D296D2CA
:1066FF00978022A2114010A228301D01B34004D26E
:10670F00978002D296800EA228301D01B34004D28A
:05671F00968002D297F4
:0F7062000266F20266F40266F80266FC0267023A
:10672400C20F74C890003AF0A20FB3B350079000A0
:106734003AE0B55F028048124D8B9000DEE0907025
:1067440071F82828738030D296802CD2968028D273
:1067540096D2978022A2114010A228301D01B34086
:1067640004D2978002D296800EA228301D01B34035
:0767740004D2968002D297C7
:0F70710002674902674B02674F02675302675974
:10677B0074C890003AF0C20F90003CE0B55F028005
:10678B0003026824A2104072900006E0FEA3E0FF13
:10679B00EF4E6021AE56AF57900006E0FCA3E0FD34
:1067AB0012000374068E048F05FF12778290000689
:1067BB00ECF0A3EDF090003DE0601A900006E0FED7
:1067CB00A3E0FFAC56AD57EF2DFDEE3CFC90000661
:1067DB00ECF0A3EDF090003DE0D39401401A900053
:1067EB0006E0FEA3E0FFAC56AD57EF2DFDEE3CFCF3
:1067FB00900006ECF0A3EDF0D210AE54AF55900024
:10680B0006E0FCA3E0FDEFC39DEE9C400CC296C2DC
:10681B0097744690003CF0C210A210B3B35007908F
:10682B00003CE0B55F02800CC296C29774469000A4
:10683B003CF0C21090003EE0B55F02800302691C81
:10684B00A2124072900002E0FEA3E0FFEF4E602127
:10685B00AE56AF57900002E0FCA3E0FD12000374AC
:10686B00068E048F05FF127782900002ECF0A3EDE9
:10687B00F090003FE0601A900002E0FEA3E0FFAC56
:10688B0056AD57EF2DFDEE3CFC900002ECF0A3ED66
:10689B00F090003FE0D39401401A900002E0FEA379
:1068AB00E0FFAC56AD57EF2DFDEE3CFC900002EC3B
:1068BB00F0A3EDF0D212AE54AF55900002E0FCA362
:1068CB00E0FDEFC39DEE9C4048124D8B9000DEE047
:1068DB00907080F82828738030D296802CD29580C7
:1068EB0028D295D2A28022A2144010A229301D01D9
:1068FB00B34004D2A28002D295800EA229301D0192
:09690B00B34004D2958002D2A22F
:0F7080000268E20268E40268E80268EC0268F263
:10691400C21274C890003EF0A212B3B350079000A4
:106924003EE0B55F028048124D8B9000DEE090702F
:106934008FF82828738030D296802CD2958028D264
:1069440095D2A28022A2144010A229301D01B34086
:1069540004D2A28002D295800EA229301D01B34038
:0769640004D2958002D2A2CB
:0F708F0002693902693B02693F0269430269499C
:10696B0074C890003EF0C212900040E0B55F028008
:10697B0003026A1DA2134072900008E0FEA3E0FF21
:10698B00EF4E6021AE56AF57900008E0FCA3E0FD40
:10699B0012000374068E048F05FF12778290000895
:1069AB00ECF0A3EDF0900041E0601A900008E0FEDF
:1069BB00A3E0FFAC56AD57EF2DFDEE3CFC9000086D
:1069CB00ECF0A3EDF0900041E0D39401401A90005D
:1069DB0008E0FEA3E0FFAC56AD57EF2DFDEE3CFCFF
:1069EB00900008ECF0A3EDF0D213AE54AF5590002D
:1069FB0008E0FCA3E0FDEFC39DEE9C40159000DE8C
:106A0B00E0B40102C296C295C2A27446900040F057
:106A1B00C213A213B3B35007900040E0B55F0280DE
:106A2B00159000DEE0B40102C296C295C2A2744674
:106A3B00900040F0C213900042E0B55F0280030269
:106A4B006B1EA2154072900004E0FEA3E0FFEF4E18
:106A5B006021AE56AF57900004E0FCA3E0FD12009E
:106A6B000374068E048F05FF127782900004ECF0FE
:106A7B00A3EDF0900043E0601A900004E0FEA3E069
:106A8B00FFAC56AD57EF2DFDEE3CFC900004ECF047
:106A9B00A3EDF0900043E0D39401401A900004E082
:106AAB00FEA3E0FFAC56AD57EF2DFDEE3CFC900086
:106ABB0004ECF0A3EDF0D215AE54AF55900004E00A
:106ACB00FCA3E0FDEFC39DEE9C4048124D8B900064
:106ADB00DEE090709EF82828738030D296802CD2FE
:106AEB00A08028D2A0D2A18022A2174010A22A30C7
:106AFB001D01B34004D2A18002D2A0800EA22A3085
:0B6B0B001D01B34004D2A08002D2A103
:0F709E00026AE4026AE6026AEA026AEE026AF431
:106B1600C21574C8900042F0A215B3B35007900096
:106B260042E0B55F028048124D8B9000DEE0907027
:106B3600ADF82828738030D296802CD2A08028D237
:106B4600A0D2A18022A2174010A22A301D01B34074
:106B560004D2A18002D2A0800EA22A301D01B34029
:076B660004D2A08002D2A1BD
:0F70AD00026B3B026B3D026B41026B45026B4B6A
:106B6D0074C8900042F0C215900044E0B55F0280F9
:106B7D0003026C1FA216407290000AE0FEA3E0FF14
:106B8D00EF4E6021AE56AF5790000AE0FCA3E0FD3A
:106B9D0012000374068E048F05FF12778290000A8F
:106BAD00ECF0A3EDF0900045E0601A90000AE0FED5
:106BBD00A3E0FFAC56AD57EF2DFDEE3CFC90000A67
:106BCD00ECF0A3EDF0900045E0D39401401A900055
:106BDD000AE0FEA3E0FFAC56AD57EF2DFDEE3CFCF9
:106BED0090000AECF0A3EDF0D216AE54AF55900024
:106BFD000AE0FCA3E0FDEFC39DEE9C40159000DE86
:106C0D00E0B40102C296C2A0C2A17446900044F045
:106C1D00C216A216B3B35007900044E0B55F0280D0
:106C2D00159000DEE0B40102C296C2A0C2A1744666
:106C3D00900044F0C2169000E0E0B402028003021E
:106C4D006D6B900074E0D395675064900074E0F420
:106C5D00042567FE9000E3E08E00F5F0E884FF7EEA
:106C6D00008F74EFC39410500CEF8574F0A4FDAC3D
:106C7D00F08D7480037574FF900074E0D3957440AB
:106C8D000B900074E0C39574F572800375720090DB
:106C9D0000FEE0D3957240069000FEE0F572900084
:106CAD00FFE0C3957250069000FFE0F57280719081
:106CBD000074E0C39567FE9000E3E08E00F5F0E808
:106CCD0084FF7E008F74EFC39410500CEF8574F029
:106CDD00A4FDACF08D7480037574FF85745B755ADB
:106CED0000900074E0255BFFAE5A50010E8E5A8F56
:106CFD005B74FFBE0009D39F4005855B72800375F1
:106D0D0072FF9000FEE0D3957240069000FEE0F514
:106D1D00729000FFE0C3957250069000FFE0F5728F
:106D2D00A204B3B3500D900075E0FE9000EBE0D3DC
:106D3D009E5002800E7407900054F0E5B554BFF5D7
:106D4D00B5801B75A710E5CDC395724008E5B55408
:106D5D00BFF5B58006E5B54440F5B575A7009000C3
:106D6D00FBE0605E900105E0A852B8000495535019
:106D7D0017900104E0A852B8000ED3955340099026
:106D8D000106E0D395624002801D75A710E5CDC3C5
:106D9D0094BF4008E5B554EFF5B58006E5B5441050
:106DAD00F5B575A700801B75A710E5CDC3944040C0
:106DBD0008E5B554EFF5B58006E5B54410F5B575A4
:106DCD00A7009000FCE0605E900108E0A852B800BA
:106DDD000495535017900107E0A852B8000ED395B3
:106DED00534009900109E0D395624002801D75A7BB
:106DFD0010E5CDC394BF4008E5B554DFF5B5800669
:106E0D00E5B54420F5B575A700801B75A710E5CD38
:106E1D00C394404008E5B554DFF5B58006E5B544AB
:106E2D0020F5B575A700E570C39413501DE5707579
:106E3D00F00284AFF07E00EF4E70051232FC800A36
:106E4D00A2EDB34005C2ED1232FCAE54AF55741035
:106E5D00C39F74279E400C900073E0C3945A400367
:106E6D00026FD5A209B340091248B37406900054BD
:106E7D00F0A20BB3500EE562D394334007E562C325
:106E8D0094CC40028041900110E0B40214121281A2
:106E9D00900077E075F05EA4FFAEF08E5C8F5D80A4
:106EAD000F90008CE075F05EA4FFAEF08E5C8F5DF0
:106EBD00E55D455C6011E5B54401F5B5742B9000B9
:106ECD0072F0124CFAD20B900073E0D3940140078C
:106EDD00E562C3941A40028002C20B9006CFE060B7
:106EED0006750801122E4F9006D3E0600675080254
:106EFD00122E4F9006D7E06006750803122E4F90A4
:106F0D0006DBE06006750804122E4F9006DFE06088
:106F1D0006750805122E4F9006E3E060067508060B
:106F2D00122E4F9006E7E06006750807122E4F905F
:106F3D0006EBE06006750808122E4F9006EFE06034
:106F4D0006750809122E4F900073E0C3945A501025
:106F5D00E570B41309900073E004F0757000803F84
:106F6D00E570B41303757000C28E758D00758B00BE
:106F7D00756500755501755400D28E900072E0C391
:106F8D0094415008900072E004F080067441900026
:106F9D0072F0900072E0B44106E5B554FEF5B5907F
:106FAD000073E0D394014007E56BC3944140028028
:106FBD0006740E900054F090089FE0600690010D4D
:0B6FCD00E060028003120BD70252E6C6
:1070E6000000010001400160018001A001C001E033
:1070F60002000300039603B603D603F4040005005A
:107106000512052405360548055A056C057E0590C9
:1071160005A805C005DE0600061406280646066E06
:1071260006AE05CF06EE00FF013F015F017F019F1E
:1071360001BF01DF01FF02FF039503B503D503F38A
:1071460003FF04FF05110523053505470559056BA2
:10715600057D058F05A705BF05CE05F10613062794
:107166000645066D06AD06ED05DD06FF0FAA0FA561
:107176000F9F0F9A0F940F8D0F870F800F780F7147
:107186000F680F600F570F4E0F450F3B0F300F253F
:107196000F1A0F0E0F020EF50EE80EDB0ECC0EBE0A
:1071A6000EAE0E9F0E8E0E7D0E6C0E5A0E470E34D0
:1071B6000E200E0C0DF70DE20DCB0DB50D9D0D85B8
:1071C6000D6D0D540D3A0D200D050CE90CCE0CB1CC
:1071D6000C940C760C580C3A0C1B0BFB0BDB0BBB04
:1071E6000B9A0B790B570B350B130AF10ACE0AAB28
:1071F6000A870A640A400A1C09F809D409B0098CEE
:1072060009670943091F08FB08D608B2088E086AF1
:107216000846082307FF07DC07B9079607730751D7
:10722600072F070D06EC06CA06AA0689066906494F
:10723600062A060A05EC05CD05B005920575055822
:10724600053C0520050504EA04CF04B5049C048228
:107256000469045104390422040B03F403DE03C851
:1072660003B2039D038903750361034D033B0328A2
:107276000316030402F202E102D102C002B002A028
:10728600029102820273026502570249023C022FF2
:1072960002220216020901FD01F201E601DB01D01C
:1072A60001C601BB01B101A7019D0194018B0182B9
:1072B60001790170016801600158015001480141DE
:1072C60001390132012B0125011E01180111010BA3
:1072D600010500FF00FA0FA60FA00F990F920F8B62
:1072E6000F840F7C0F740F6B0F620F580F4E0F43F6
:1072F6000F380F2C0F1F0F120F050EF70EE80ED8C2
:107306000EC80EB70EA50E930E800E6C0E580E42CA
:107316000E2C0E150DFD0DE40DCB0DB10D950D7951
:107326000D5D0D3F0D200D010CE10CC00C9E0C7C7B
:107336000C590C350C100BEA0BC40B9E0B760B4F3D
:107346000B260AFD0AD40AAA0A800A550A2A09FF48
:1073560009D409A8097C0950092508F908CD08A10E
:107366000875084A081E07F307C8079D07730749EB
:10737600072006F706CE06A6067E06570630060A3C
:1073860005E405BF059B057705540532051004EF96
:1073960004CE04AE048F047104530435041903FDAE
:1073A60003E203C703AD0394037B0363034B033478
:1073B600031E030802F302DE02CA02B602A302910A
:1073C600027F026D025C024C023C022C021D020E80
:1073D600020001F201E401D701CA01BE01B101A612
:1073E600019A018F0185017A01700166015D0153E1
:1073F600014A014101390131012901210119011215
:10740600010B010400FD00F700F000EA00E400DED5
:1074160000D900D300CE00C900C400BF00BA00B531
:1074260000B100AD00A800A400A0009C0099009542
:107436000091008E008A008700840081007E007B18
:10009E0075B50075840175A70075FFA075EF069004
:1000AE000050E4F075C91075A70F75A1C775A700AC
:1000BE0075D90075CE0C75A70F75F1FE75F2FF752B
:1000CE00F30775F47875A4BA75A5FF75A60775AE16
:1000DE000075AFFF75D48175D5FF75D6FF75D7FF47
:1000EE0075A70075A20175A14775F8092275E60876
:1000FE0075E71075BC0175BE0475BD6C75BE0775D0
:10010E00BDA075BE0875BD0175BC0075BB1875BC6C
:10011E002075BA0875E88075D11375A70F75E105BE
:10012E0075E20075C7401248B375970075978074D5
:10013E000A1277727597C0E5975420700280F87591
:10014E008F0275A700D2AF75980075A90C75A70F11
:10015E0075AB4375ADFB75AC1E75A71075C91875DB
:10016E00CA0075CB0075C80475A700758912758E07
:10017E0004758C00758A00C2A9D28C758D00758BA2
:10018E0000D2ABD28E75B62075D944C2992290009A
:10019E008AE090089EF0900095E090089FF0900005
:1001AE0096E09008A0F09000B5E09008A1F09000C5
:1001BE00C2E09008A2F09000D0E09008A3F090006A
:1001CE00DEE09008A4F09000E0E09008A5F090002A
:1001DE00EEE09008A6F09000FBE09008A7F09000EB
:1001EE00FCE09008A8F090010EE09008A9F09001B4
:1001FE0026E09008ABF0900174E09008ACF090010E
:10020E0075E09008ADF0900176E09008AEF09001A8
:10021E000DE09008AFF09000F7E09008B0F090007D
:10022E00AEE09008B1F09000AFE09008B2F0900010
:10023E00A9E09008B3F09000AAE09008B4F0900105
:10024E0013E09008B5F0900114E09008B6F090011C
:10025E0015E09008B7F0900116E09008B8F0900104
:10026E0017E09008B9F09006CEE09008BAF090062C
:10027E00D2E09008BBF09006D6E09008BCF0900655
:10028E00DAE09008BDF09006DEE09008BEF0900631
:10029E00E2E09008BFF09006E6E09008C0F090060D
:1002AE00EAE09008C1F09006EEE09008C2F09006E9
:1002BE00F2E09008C3F0900776E09008C4F0900743
:1002CE0077E09008C5F0900778E09008C6F09007A8
:1002DE0079E09008C7F090077AE09008C8F0900790
:1002EE007BE09008C9F090077CE09008CAF0900778
:1002FE007DE09008CBF090077EE09008CCF0900760
:10030E007FE09008CDF0900780E09008CEF0900747
:10031E0081E09008CFF0900782E09008D0F090072F
:10032E0083E09008D1F0900784E09008D2F0900717
:10033E0085E09008D3F0900786E09008D4F0900105
:10034E0018E09008D5F0900119E09008D6F09001D1
:10035E001AE09008D7F090011BE09008D8F09001B9
:10036E001CE09008D9F090011DE09008DAF09001A1
:10037E001EE09008DBF090011FE09008DCF0900189
:10038E0020E09008DDF0900121E09008DEF0900072
:10039E00BCE09008DFF09000F4E09008E0F09001EF
:1003AE002CE09008E1F090012DE09008E2F0229010
:1003BE00089EE090008AF090089FE0900095F090E3
:1003CE0008A0E0900096F09008A1E09000B5F090A3
:1003DE0008A2E09000C2F09008A3E09000D0F09048
:1003EE0008A4E09000DEF09008A5E09000E0F09008
:1003FE0008A6E09000EEF09008A7E09000FBF090C9
:10040E0008A8E09000FCF09008A9E090010EF09092
:10041E0008ABE0900126F09008AFE090010DF0904F
:10042E0008B0E09000F7F09008B1E09000AEF090C8
:10043E0008B2E09000AFF09008B3E09000A9F09001
:10044E0008B4E09000AAF09008B5E0900113F09087
:10045E0008B6E0900114F09008B7E0900115F09006
:10046E0008B8E0900116F09008B9E0900117F090EE
:10047E0008BAE09006CEF09008BBE09006D2F0905D
:10048E0008BCE09006D6F09008BDE09006DAF09039
:10049E0008BEE09006DEF09008BFE09006E2F09015
:1004AE0008C0E09006E6F09008C1E09006EAF090F1
:1004BE0008C2E09006EEF09008C3E09006F2F090CD
:1004CE0008C4E0900776F09008C5E0900777F090AA
:1004DE0008C6E0900778F09008C7E0900779F09092
:1004EE0008C8E090077AF09008C9E090077BF0907A
:1004FE0008CAE090077CF09008CBE090077DF09062
:10050E0008CCE090077EF09008CDE090077FF09049
:10051E0008CEE0900780F09008CFE0900781F09031
:10052E0008D0E0900782F09008D1E0900783F09019
:10053E0008D2E0900784F09008D3E0900785F09001
:10054E0008D4E0900786F09008D5E0900118F0905E
:10055E0008D6E0900119F09008D7E090011AF090BB
:10056E0008D8E090011BF09008D9E090011CF090A3
:10057E0008DAE090011DF09008DBE090011EF0908B
:10058E0008DCE090011FF09008DDE0900120F09073
:10059E0008DEE0900121F09008DFE09000BCF090C2
:1005AE0008E0E09000F4F09008E1E090012CF0906B
:1005BE0008E2E090012DF022754800900896E4F0D4
:1005CE00A3F0753200753100754E00754F00C22FC5
:1005DE00D23090089FE06002D22474FE900898F802
:1005EE00E4F0E8A3F074FE90089CF8E4F0E8A3F0C1
:1005FE0074FE90089AF8E4F0E8A3F0745A9008F0AC
:10060E00F0745A9008F1F0D231C22DC233C232C208
:10061E002EC235C23B22750B00750A00AE0AAF0B17
:10062E00AC08AD09EDC39FEC9E401674FF127772B5
:10063E0075CF01780B740126F6500418E436F65087
:10064E00DB22C2AF75D904758F0375B7A575B7F1E7
:10065E0090F800E4F0758F0175B7A575B7F1E52830
:10066E0090F800F075B7A575B7F190F801E4F07544
:10067E00B7A575B7F19008E4E090F802F075B7A54C
:10068E0075B7F19008E8E090F803F075B7A575B767
:10069E00F19008E5E090F804F075B7A575B7F19004
:1006AE0008E6E090F805F075B7A575B7F19008E784
:1006BE00E090F806F075B7A575B7F19008E9E090EF
:1006CE00F807F0758F0075D944D2AF22900050E034
:1006DE00B4AB61C2AF75D90475B62275F522758FAC
:1006EE000375B7A575B7F1740090F600F0758F011C
:1006FE00755B00755A00AE5AAF5B7445BE00279FFE
:10070E00402475B7A575B7F190089E120048E0FC1D
:10071E0090F600120048ECF0785B740126F6500457
:10072E0018E436F650D0758F0075F51175B6207534
:10073E00D944D2AF22C2AF75F52275D904755B00CC
:10074E00755A00AE5AAF5B7445BE00229F401F9093
:10075E00F600120048E493FC90089E120048ECF05C
:10076E00785B740126F6500418E436F650D575D928
:10077E004475F511D2AF22900050E0B4AA02800366
:10078E000208C2C2AF75D90475B62275F522758FEF
:10079E000375B7A575B7F1740090F400F075B7A5A1
:1007AE0075B7F1740090F200F075B7A575B7F174D6
:1007BE000090F000F075B7A575B7F1740090EE00DB
:1007CE00F0758F01755B00755A00AE5AAF5B74FF02
:1007DE00C39F74019E402475B7A575B7F19000882C
:1007EE00120048E0FC90F400120048ECF0785B74C4
:1007FE000126F6500418E436F650CF755B00755A94
:10080E0000AE5AAF5B74FFC39F74019E402475B750
:10081E00A575B7F1900288120048E0FC90F2001224
:10082E000048ECF0785B740126F6500418E436F6B6
:10083E0050CF755B00755A00AE5AAF5B74FFC39F05
:10084E0074019E402475B7A575B7F1900488120007
:10085E0048E0FC90F000120048ECF0785B74012642
:10086E00F6500418E436F650CF755B00755A00AE9C
:10087E005AAF5B74FFC39F74019E402475B7A57574
:10088E00B7F1900688120048E0FC90EE0012004886
:10089E00ECF0785B740126F6500418E436F650CF6F
:1008AE00758F0075F51175B62075D944D2AF743AAF
:1008BE00900788F022900050E0B4AA028003020A4A
:1008CE0000C2AF75D90475B62275F522758F037502
:1008DE00B7A575B7F1740090EC00F075B7A575B7B4
:1008EE00F1740090EA00F075B7A575B7F174009039
:1008FE00E800F075B7A575B7F1740090E600F075D5
:10090E008F01755B00755A00AE5AAF5B74FFC39FC3
:10091E0074019E402475B7A575B7F190008812003A
:10092E0048E0FC90EC00120048ECF0785B74012675
:10093E00F6500418E436F650CF755B00755A00AECB
:10094E005AAF5B74FFC39F74019E402475B7A575A3
:10095E00B7F1900288120048E0FC90EA00120048BD
:10096E00ECF0785B740126F6500418E436F650CF9E
:10097E00755B00755A00AE5AAF5B74FFC39F74016E
:10098E009E402475B7A575B7F1900488120048E013
:10099E00FC90E800120048ECF0785B740126F650EB
:1009AE000418E436F650CF755B00755A00AE5AAF98
:1009BE005B74FFC39F74019E402475B7A575B7F194
:1009CE00900688120048E0FC90E600120048ECF019
:1009DE00785B740126F6500418E436F650CF758F06
:1009EE000075F51175B62075D944D2AF743A9007DB
:1009FE0088F022C2AF75D90475F522755B00755A61
:100A0E0000AE5AAF5B74FFC39F74019E401F90F4FB
:100A1E0000120048E493FC900088120048ECF07835
:100A2E005B740126F6500418E436F650D4755B005C
:100A3E00755A00AE5AAF5B74FFC39F74019E401F80
:100A4E0090F200120048E493FC900288120048ECE9
:100A5E00F0785B740126F6500418E436F650D4751F
:100A6E005B00755A00AE5AAF5B74FFC39F74019E54
:100A7E00401F90F000120048E493FC90048812008E
:100A8E0048ECF0785B740126F6500418E436F65004
:100A9E00D4755B00755A00AE5AAF5B74FFC39F747A
:100AAE00019E401F90EE00120048E493FC900688D1
:100ABE00120048ECF0785B740126F6500418E43608
:100ACE00F650D475F51175D944D2AF74019000D19A
:100ADE00F0743A900788F09008F77401F022C2AFD4
:100AEE0075D90475F522755B00755A00AE5AAF5B69
:100AFE0074FFC39F74019E401F90EC00120048E4E7
:100B0E0093FC900088120048ECF0785B740126F696
:100B1E00500418E436F650D4755B00755A00AE5A80
:100B2E00AF5B74FFC39F74019E401F90EA001200DA
:100B3E0048E493FC900288120048ECF0785B740154
:100B4E0026F6500418E436F650D4755B00755A003C
:100B5E00AE5AAF5B74FFC39F74019E401F90E800B6
:100B6E00120048E493FC900488120048ECF0785B85
:100B7E00740126F6500418E436F650D4755B0075F1
:100B8E005A00AE5AAF5B74FFC39F74019E401F9014
:100B9E00E600120048E493FC900688120048ECF040
:100BAE00785B740126F6500418E436F650D475F5C9
:100BBE001175D944D2AF74029000D1F0743A9007F7
:100BCE0088F074029008F7F02274019000D1F09032
:100BDE00089FE0903CBBF828287380188016A2A3CB
:100BEE00400674029000D1F0800AA2A4400674025E
:040BFE009000D1F0A2
:0C3CBB00020BE8020BEA020BEC020BF813
:100C02009000D1E0B40105A239B34002801AD23972
:100C12001248B3120A0174019000D1F01203BD12FE
:100C22003EE8741B900054F09000D1E0B40206A29A
:100C320039B3B34002801AC2391248B3120AEC74B3
:100C4200029000D1F01203BD123EE8741B900054D2
:100C5200F022E54F64046006E59964FF600280318A
:100C6200A22F4004D22F8027E54F600874E6254F5B
:100C7200900054F0E54E600874F0254E900054F058
:100C8200E54FB4010280FE754F00754E00C22F8001
:100C920002C22FE54F903CC7F8282873754F00E534
:100CA20099B4FF03754E01E599B4FE03754E02E552
:100CB20099B4FD03754E03E599B4FC03754E04E542
:100CC20099B4FA03754E05E599B4FB06754F011206
:100CD20048B3E599B4F906754F041248B3E599B4DF
:100CE200F7331248B3C29C74AB900050F01206DA8C
:100CF20074AA900050F09008F7E0B401051207853D
:100D020080031208C3900050E4F0D29C754F007526
:100D12004E007599F7E599D394E54007E599C39498
:100D2200F040028016859950754F027E017F00E5E2
:100D320050C394E61277928E338F34900896E4F083
:100D4200A3F0E599D394C24007E599C394E6400223
:100D52008028859950754F0374E5C39550F5347515
:100D62003300AE33AF349070E6127761E493F874D7
:100D72000193900896C8F0A3C8F0D2990210DF90B0
:100D820008ABE0700AA225B35005A226B340028048
:100D92005C900896E0FEA3E0FF74FFBE00039F5044
:100DA20009EFC39446EE9406402B900896E0FEA30A
:100DB200E0FFEFD3946DEE94064009EFC394EEEE9C
:100DC20094064011900896E0FEA3E0FFEFD394FF53
:100DD200EE94064013900896E0FEA3E0FF90008890
:100DE200120048E599F08003859975801190089664
:100DF200E0FEA3E0FF900088120048E599F0900819
:100E0200961277A0900896E0FEA3E0FFEFB40106E9
:100E1200EEB407028003020EDA900788E0B43C02C7
:100E22008003020EDAA225B35005A226B340028047
:100E320055C29C1203BD900095E09008F6F0124056
:100E420061900174E09008ACF0900175E09008ADFB
:100E5200F0900176E09008AEF074AB900050F01282
:100E620006DA74AA900050F09008F7E0B401051277
:100E7200078580031208C39008F7E09000D1F09034
:100E82000050E4F08047C29C12019C74009008ACB0
:100E9200F074009008ADF074009008AEF0900095E8
:100EA200E09008F6F012406174AB900050F0120628
:100EB200DA74AA900050F01207851208C3D29C750A
:100EC20099FB75096475080012062480FED29C7590
:100ED2004F00754E007599FB0210DF900896E0FEF8
:100EE200A3E0FFEF4E7006859932753100900896A7
:100EF200E0FEA3E0FF74016F4E701BAC31AD32AA6D
:100F020033AB34ED2BFBEC3AFA8A068B0790008860
:100F1200120048E599F09008961277A0900896E0A2
:100F2200FEA3E0FF74026F4E7021AC31AD327456F5
:100F32006D4C7006E55064E6600280031248B312FD
:100F42004061855099754F00754E000210DF900880
:100F520096E0FEA3E0FF900088120048E599F09029
:100F620008961277A0900896E0FEA3E0FFAC33AD9E
:100F7200348F028E038C068D0790712C127761E4F8
:100F820093F9740193FEEAD39EEB99400985509937
:100F9200754F00754E000210DF900896E0FEA3E048
:100FA200FF900088120048E599F09008961277A009
:100FB200900896E0FEA3E0FFEFB40006EEB4010253
:100FC20080030210DF900066E0D394C7400B9000CC
:100FD20066E0C394C8F551801A900066E0D394632A
:100FE200400B900066E0C39464F551800690006661
:100FF200E0F551E55175F002A4FFAEF08F74EF9069
:1010020000881277C3EFFCE0FDEC90008B1277C3EF
:10101200EDFCE0FDEC2DB5510280030210D10FEF83
:101022009000881277C3E574FFE0FCEF90008C1209
:1010320077C3ECFFE0FCEFC39CB5510280030210C2
:10104200D1E57490008A1277C3E574FFE0FCEF905B
:10105200008D1277C3ECFFE0FCEF2CB55171E57403
:1010620090008E1277C3E0C395519008E4F0E574C6
:1010720090008F1277C3E0C395519008E5F0E574B4
:101082009000921277C3E0C395519008E6F0E574A0
:101092009000931277C3E0C395519008E7F0E5748E
:1010A2009000941277C3E0C395519008E8F0E5747C
:1010B2009000951277C3E0C395519008E9F01206AB
:1010C200507599F975096475080012062480FE7539
:0D10D20099FF75096475080012062480FE60
:0F3CC700020C9E020D81020EDD020F50020F9BB8
:1010DF0022E54E903CD6F82828730211C49008964A
:1010EF00E0FEA3E0FF900056120048E0F59990084B
:1010FF00961277A0900896E0FEA3E0FF741C6F4E47
:10110F007003754E000211C4856F990211C49008C7
:10111F0096E0FEA3E0FF900088120048E0F599EFFB
:10112F00B40107EEB40703754E009008961277A02E
:07113F000211C4900897E0C3
:0F3CD6000210E90210EC02111702111D02114237
:10114600903D48F828287385539980678560998073
:1011560062856299805D8566998058856899805315
:10116600856999804E856A998049856B99804490F6
:10117600001BE0F599803CA230B340077599FAC28E
:10118600308017A224B3400575990F800B90005448
:10119600E0F599900054E4F0C2248017856C99809C
:1011A60012856799800D856D9980087599FC800375
:0311B600754E0073
:103D480002114D02115202115702115C0211610257
:103D5800116602116B02117002117502117D0211B8
:0D3D6800A20211A70211AC0211B10211B6A6
:0B11B9009008961277A08003123F43BD
:033CE5000211C108
:1011C40022E538255BFFAE5A50010E9000881200CC
:1011D40048E0F539E538255BFFAE5A50010E0FBFE4
:1011E40000010E900088120048E0F53A85403CE585
:1011F40039B53A058539388041E53AD39539401DEA
:10120400E53AC39539853BF0A4FFAEF0E53C8E0486
:101214008F05FF127782ED2539F538801DE539C336
:10122400953A853BF0A4FFAEF0E53C8E048F05FFB4
:10123400127782EDF4042539F53822E53AD395394D
:10124400401DE53AC39539853BF0A4FFAEF0E53C7B
:101254008E048F05FF127782ED2539F538801DE560
:1012640039C3953A853BF0A4FFAEF0E53C8E048F7C
:1012740005FF127782EDF4042539F5382290008EAB
:10128400E0B4017FE56875F00A84FF7E008F38E5DD
:101294006875F00A84ADF07C008D3B75400A755A80
:1012A40005755B24E538C3941150051211C58006F9
:1012B4009005BDE0F538E538C394F05008E5389062
:1012C4000077F0800674EF900077F0E56875F00A17
:1012D40084FF7E008F38E56875F00A84ADF07C00E9
:1012E4008D3B75400A755A05755B5AE538C39411F0
:1012F40050051211C580069005F3E0F538E53890E5
:10130400004FF02290008EE0B40102800302139695
:10131400E56875F00A84FF7E008F38E56875F00A89
:1013240084ADF07C008D3B75400A755A05755B36BB
:10133400E538C3941150051211C580069005CFE01D
:10134400F538E538C394F0500585384C8003754C66
:10135400EFE56875F00A84FF7E008F38E56875F064
:101364000A84ADF07C008D3B75400A755A05755BA7
:1013740048E538C3941150051211C580069005E163
:10138400E0F538E538C394F0500585384D80037591
:101394004DEF22E56075F00484FF7E008F38E56030
:1013A40075F00484ADF07C008D3B754004755A01E2
:1013B400755B00E538C3943F50051211C580069053
:1013C40001C7E0F538E538900890F8E4F0E8A3F0B8
:1013D400900053E075F020A4FFAEF09000D9E08EA9
:1013E400048F05FF1277828D389000C1E0D3956099
:1013F40050030214A29000E5E0D395604010ED90F4
:1014040001C81277C3E0F52C752B0002149F9000DD
:10141400B0E0D395604043E5389001C81277C3E04B
:10142400F539E5389001E81277C3E0F53A9000E524
:10143400E0F4042560F53B9000B0E0FE9000E5E0A8
:10144400F4042EF53CE539B53A05853938800312A4
:10145400123F85382C752B008041E5389001E81245
:1014640077C3E0F539E5389002081277C3E0F53A1E
:101474009000B0E0F4042560F53B9000C1E0FE90DC
:1014840000B0E0F4042EF53CE539B53A0585393869
:10149400800312123F85382C752B000215499000E9
:1014A400E8E0D395605011E5389002481277C3E024
:1014B400F52C752B000215499000B1E0D3956050CE
:1014C40043E5389002281277C3E0F539E5389002F5
:1014D400481277C3E0F53A9000B1E0F4042560F5D2
:1014E4003B9000E8E0FE9000B1E0F4042EF53CE50A
:1014F40039B53A05853938800312123F85382C7581
:101504002B008041E5389002081277C3E0F539E5F5
:10151400389002281277C3E0F53A9000C1E0F40451
:101524002560F53B9000B1E0FE9000C1E0F4042E8C
:10153400F53CE539B53A05853938800312123F8503
:10154400382C752B00229000F9E0F53D754011759B
:101554005A02755B00AE52AF53E53D75F00FA4FD22
:10156400ACF0EDD39FEC9E4021E53D8E048F05FF4A
:10157400127782ED75F010A4FFAEF0E56075F011FE
:1015840084FD7C00ED2FF53E800EE56075F011843E
:10159400FF7E00EF24F0F53E853E38E56075F011DE
:1015A40084AFF07E008F3B1211C585383FAE52AF39
:1015B400539000F9E075F00FA4FDACF0EDD39FEC6F
:1015C4009E4028755A02755B10853E381211C585F8
:1015D4003F3985383AAE52AF53E53D8E048F05FF4F
:1015E4001277AD8D3B853D3C12123FE53890089053
:1015F400F8E4F0E8A3F0752C64752B00229000F950
:10160400E0F53D754011755A02755B00AE52AF535B
:10161400E53D75F00FA4FDACF0EDD39FEC9E4021A9
:10162400E53D8E048F05FF127782ED75F010A4FF5F
:10163400AEF0E56275F01184FD7C00ED2FF53E807F
:101644000EE56275F01184FF7E00EF24F0F53E850F
:101654003E38E56275F01184AFF07E008F3B1211C5
:10166400C585383FAE52AF539000F9E075F00FA432
:10167400FDACF0EDD39FEC9E4028755A02755B10CB
:10168400853E381211C5853F3985383AAE52AF537D
:10169400E53D8E048F05FF1277AD8D3B853D3C12F1
:1016A400123FE538900890F8E4F0E8A3F0E56C60A8
:1016B40017E56CC394FE50109000EDE0B40209905D
:1016C40000DBE0D3940B5002801F900890E0FEA34F
:1016D400E0FFE56C12779274E78E048F05FF1277B2
:1016E40082900890ECF0A3EDF09000C3E0B4045FA6
:1016F400E56075F00484FF7E008F38E56075F004C2
:1017040084ADF07C008D3B754004755A01755B0017
:10171400E538C3943F50051211C580069001C7E017
:10172400F538900890E0FEA3E0FFE5381277927454
:10173400328E048F05FF127782900890E0FEA3E0BA
:10174400FFEF2DFDEE3CFC900890ECF0A3EDF0755E
:101754002C64752B002290008EE0B40146E5687578
:10176400F00A84FF7E008F38E56875F00A84ADF0D6
:101774007C008D3B75400A755A05755B00E538C3DE
:10178400941150051211C58006900599E0F538AE04
:101794002BAF2CE5382FFF50010E74641277D58ED1
:1017A4002B8F2C90008FE0B40146E56975F00A8414
:1017B400FF7E008F38E56975F00A84ADF07C008DFA
:1017C4003B75400A755A05755B6CE538C394115036
:1017D400051211C58006900605E0F538AE2BAF2C36
:1017E400E5382FFF50010E74641277D58E2B8F2CA1
:1017F40090009EE0B40249E56BC3944175F0058402
:10180400FF7E008F38E56B75F00584ADF07C008DAC
:101814003B754005755A06755B00E538C394135053
:10182400051211C5800690069BE0F538AE2BAF2C4F
:10183400E5382FFF50010E74641277D58E2B8F2C50
:101844009000E0E0B4020280030218F9E56075F04C
:101854001584FF7E008F38E56075F01584ADF07C4B
:10186400008D3B754015755A03755BF4E538C394D8
:101874000B50051211C58006900487E0F538E53851
:1018840075F0FFA4FFAEF09000E1E08E048F05FF39
:10189400127782ED900074F0E56775F078A4FFAEDE
:1018A400F074FF8E048F05FF1277828C5A8D5B745F
:1018B400028C068D071200398F38AC5AAD5B740464
:1018C400FF1277AD8D3B754004755A06755B28E5AC
:1018D40038C3941D50051211C580069006CDE0F55D
:1018E40038AE2BAF2CE5382FFF50010E74641277FD
:1018F400D58E2B8F2C90008DE0B4025DE56275F0DF
:1019040064A4FFAEF074081200398E5C8F5D740518
:101914008E048F05FF1277828D38AE5CAF5D74053F
:101924008E048F05FF1277AD8D3B754005755A0502
:10193400755BDEE538C3941350051211C58006901B
:101944000679E0F538AE2BAF2CE5382FFF50010EA9
:1019540074641277D58E2B8F2C9000CFE0707F901B
:101964000053E075F00A84FF7E008F38900053E046
:1019740075F00A84ADF07C008D3B75400A755A05FC
:10198400755BC0E538C3940E50051211C5800690EE
:101994000656E0F538E538900078F09000EEE0B4B3
:1019A400023C900053E075F00A84FF7E008F38906B
:1019B4000053E075F00A84ADF07C008D3B75400A5D
:1019C400755A05755BCFE538C3940E50051211C5E1
:1019D4008006900665E0F538E538900079F02290AD
:1019E4000096E0B401179008EBE0252CFFAE2B50D5
:1019F400010E9000EAE01277D58E2B8F2C90010E09
:101A0400E0B4011490010FE0A852B80004955350BB
:101A140007E560C39561400280139000B8E0252C6F
:101A2400FFAE2B50010E8E2B8F2C021E4A90009677
:101A3400E0B40306A22DB3B3400280509008F5E051
:101A440070109008EEE0C39405A852B800069553B0
:101A5400400280109000B8E0252CFFAE2B50010E00
:101A64008E2B8F2C9008F5E0600D9008EEE0A852C4
:101A7400B800069553400280109000B8E0252CFF72
:101A8400AE2B50010E8E2B8F2C021E4A900090E03C
:101A9400B402028003021E4A900093E0602FE568BE
:101AA400D394464028900012E0FEA3E0FF9000CEBD
:101AB400E075F003A4FDACF0EFD39DEE9C400E90D6
:101AC40000F2E0A852B80005D395535003021E4A11
:101AD4009000C3E0B403028003021C9285625B752C
:101AE4005A0090009AE0A852B800049553500E9002
:101AF400009BE0A85AB80005D3955B5003021C8FE5
:101B0400E56275F002A4FFAEF074158E048F05FF34
:101B14001277828C068D07900618120048FEE0FFAB
:101B2400EE900092E0FEEF8E0088F0A4FFAEF07419
:101B3400648E048F05FF1277828C5A8D5B9000535C
:101B4400E075F018A4FFAEF09000D9E08E048F0584
:101B5400FF1277828C068D07900630120048AE5A29
:101B6400AF5BE012779274648E048F05FF12778264
:101B74008C5A8D5BE566A85AB80005D3955B500373
:101B8400021C06E566C3955BFFE4955AFE8E5A8FE8
:101B94005B7428BE00039F500C755B28755A007453
:101BA4000D900054F0AE5AAF5B900093E012779220
:101BB40074288E048F05FF1277828C5A8D5B9008EF
:101BC40090E0FEA3E0FF740A8E048F05FF12778273
:101BD4008D068C07AC5AAD5BCFCECF120003740ACE
:101BE4008E048F05FF1277828C5A8D5B900890E0EB
:101BF400FEA3E0FF1277DD900890EEF0A3EFF00271
:101C04001C8FE566A85AB80004955B507EAE5AAFA7
:101C14005BE5661277D58E5A8F5B7428BE00039FEE
:101C2400500C755B28755A00740D900054F0AE5A30
:101C3400AF5B900093E012779274288E048F05FFB7
:101C44001277828C5A8D5B900890E0FEA3E0FF74BB
:101C54000A8E048F05FF1277828D068C07AC5AAD6D
:101C64005BCFCECF120003740A8E048F05FF127768
:101C7400828C5A8D5B900890E0FEA3E0FFEF2DFD6F
:101C8400EE3CFC900890ECF0A3EDF0021E4A9000AC
:101C9400DBE08560F0A4FFAEF07405127792740760
:101CA4001200398E5A8F5B90009AE0A852B8000453
:101CB4009553501290009BE075F002A4FDACF0EF38
:101CC400C39DEE9C4003021E4AE56075F00B84FF41
:101CD4007E00900618120048FEE0FFEE900092E0AD
:101CE400FEEF8E0088F0A4FFAEF074648E048F05BE
:101CF400FF1277828C5A8D5B900053E075F018A424
:101D0400FFAEF09000D9E08E048F05FF1277828C2D
:101D1400068D07900630120048AE5AAF5BE012778A
:101D24009274648E048F05FF1277828C5A8D5BE562
:101D340066A85AB80005D3955B5003021DC1E56639
:101D4400C3955BFFE4955AFE8E5A8F5B7428BE00E0
:101D5400039F500C755B28755A00740D900054F065
:101D6400AE5AAF5B900093E012779274288E048F82
:101D740005FF1277828C5A8D5B900890E0FEA3E0F9
:101D8400FF740A8E048F05FF1277828D068C07ACD0
:101D94005AAD5BCFCECF120003740A8E048F05FFB9
:101DA4001277828C5A8D5B900890E0FEA3E0FF12BC
:101DB40077DD900890EEF0A3EFF0021E4AE566A8E6
:101DC4005AB80004955B507EAE5AAF5BE566127755
:101DD400D58E5A8F5B7428BE00039F500C755B2808
:101DE400755A00740D900054F0AE5AAF5B90009396
:101DF400E012779274288E048F05FF1277828C5A32
:101E04008D5B900890E0FEA3E0FF740A8E048F05BA
:101E1400FF1277828D068C07AC5AAD5BCFCECF1202
:101E24000003740A8E048F05FF1277828C5A8D5B2F
:101E3400900890E0FEA3E0FFEF2DFDEE3CFC90083F
:101E440090ECF0A3EDF0229000EEE0B4027BE560AC
:101E540075F00884FF7E008F38E56075F00884AD66
:101E6400F07C008D3B754008755A01755BE0E538E0
:101E7400C3943F50051211C58006900287E0F538DF
:101E8400E538900892F8E4F0E8A3F0900892E0FEB8
:101E9400A3E0FFAC2BAD2C12000374648E048F05F9
:101EA400FF127782900892ECF0A3EDF090008BE0A3
:101EB4008C068D0712779274648E048F05FF127757
:101EC40082900892ECF0A3EDF0900890E0FEA3E07D
:101ED400FFAC2BAD2C12000374648E048F05FF122B
:101EE4007782900890ECF0A3EDF090008BE08C06E4
:101EF4008D0712779274648E048F05FF1277829097
:101F04000890ECF0A3EDF0A204401DAE52AF537460
:101F140005BE00039F5002D204E562D394CC40086E
:101F2400D2027411900054F0229000EDE0B4020843
:101F34009000DBE0640B60028045900890E0FEA313
:101F4400E0FFE56C12779274E78E048F05FF127739
:101F540082900890ECF0A3EDF09000EEE0B4021F44
:101F6400900892E0FEA3E0FFE56C12779274E78E8E
:101F7400048F05FF127782900892ECF0A3EDF090A5
:101F840000ADE05402601B9000A4E0A852B8001217
:101F9400D39553400DA204B3B35007E562C3949A9A
:101FA4004002805FAE35AF369000A2E075F002A427
:101FB400FDACF0EF2DFDEE3CFC74022DFD50010C48
:101FC400E562BC003ED39D403A754401A2344033DF
:101FD4009000A3E075F05EA4FDACF07405FF1277E9
:101FE400828C5C8D5D124CFA900890E0FEA3E0FFB9
:101FF4009000A3E02FFF50010E900890EEF0A3EFA5
:10200400F0D234E562A835B8000495365002C234E3
:10201400856236753500E544700302212390010082
:10202400E0C395445003022115900110E0C39402CB
:1020340040030220BFE56875F00A84FF7E00900526
:1020440088120048E0F55B755A00AE5AAF5B900009
:10205400A3E012779274648E048F05FF1277828C4A
:102064005C8D5D900100E004C395448C068D0712DD
:102074007792900100E08E048F05FF1277828C5CCA
:102084008D5D900890E0FEA3E0FFEF2DFDEE3CFC9B
:10209400900890ECF0A3EDF09000EEE0B4021A90FA
:1020A4000892E0FEA3E0FFAA5CAB5DEF2BFBEE3AE7
:1020B400FA900892EAF0A3EBF08056900100E00455
:1020C400C39544854CF0A4FFAEF0900100E08E046B
:1020D4008F05FF1277828C5C8D5D900890E0FEA3E3
:1020E400E0FFEF2DFDEE3CFC900890ECF0A3EDF04A
:1020F4009000EEE0B4021A900892E0FEA3E0FFAA7A
:102104005CAB5DEF2BFBEE3AFA900892EAF0A3EB9E
:10211400F00544900100E0C39544500375440090D9
:1021240000ADE05401601B9000A1E0A852B8001279
:10213400D39553400DA204B3B35007E560C394CCC8
:102144004002806090009FE075F003A4FFAEF0E5CC
:10215400412FFF50010E74032FFF50010EE560BEA6
:102164000042D39F403E754501A23440379000A001
:10217400E075F05EA4FFAEF074058E048F05FF12C7
:1021840077828C5C8D5D124CFA900890E0FEA3E09F
:10219400FF9000A0E02FFF50010E900890EEF0A3F6
:1021A400EFF0D234E560C395415002C234856041FA
:1021B400E54570030222BD900101E0C3954550033B
:1021C4000222AF900110E0C394024003022259E5B9
:1021D4006875F00A84FF7E00900588120048E0F5D7
:1021E4005B755A00AE5AAF5B9000A0E01277927410
:1021F400648E048F05FF1277828C5C8D5D900101E3
:10220400E004C395458C068D07127792900101E096
:102214008E048F05FF1277828C5C8D5D900890E0B0
:10222400FEA3E0FFEF2DFDEE3CFC900890ECF0A344
:10223400EDF09000EEE0B4021A900892E0FEA3E004
:10224400FFAA5CAB5DEF2BFBEE3AFA900892EAF042
:10225400A3EBF08056900101E004C39545854DF051
:10226400A4FFAEF0900101E08E048F05FF12778287
:102274008C5C8D5D900890E0FEA3E0FFEF2DFDEEF9
:102284003CFC900890ECF0A3EDF09000EEE0B4027A
:102294001A900892E0FEA3E0FFAA5CAB5DEF2BFB73
:1022A400EE3AFA900892EAF0A3EBF00545900101AA
:1022B400E0C395455003754500900890E0FEA3E007
:1022C400FF9000B2E0BE00039F500D9000B2E0907A
:1022D4000890F8E4F0E8A3F09000EEE0B402129065
:1022E4000892E0FEA3E0FF9000B2E0BE00059F402C
:1022F40002800D9000B2E0900892F8E4F0E8A3F0B8
:10230400229000EEE0B401028003022453A204B33D
:10231400500302243A9000B9E0B4017A900890E0A6
:10232400FEA3E0FFAC52AD53120003743C8E048F45
:1023340005FF1277829000C9E0BC00159D40129001
:102344000890E0FEA3E0FF9000CBE0BE00039F50A6
:1023540002D203900890E0FEA3E0FFAC52AD53120A
:102364000003743C8E048F05FF1277829000C9E04D
:10237400C3940ABC001AD39D4016900890E0FEA3B3
:10238400E0FF9000CBE0C39405BE0004D39F50024D
:102394008002C203807A900890E0FEA3E0FFAC5272
:1023A400AD5312000374788E048F05FF1277829068
:1023B40000C9E0BC00159D4012900890E0FEA3E027
:1023C400FF9000CBE0BE00039F5004D203804190F5
:1023D4000890E0FEA3E0FFAC52AD53120003747802
:1023E4008E048F05FF1277829000C9E0C3940ABC63
:1023F400001AD39D4016900890E0FEA3E0FF9000E1
:10240400CBE0C39405BE0004D39F50028002C203F4
:10241400A203B34021900890E0FEA3E0FF9000CA1D
:10242400E012779274648E048F05FF12778290080D
:1024340090ECF0A3EDF0A203B3400CA23840067474
:1024440024900054F0D238A2034002C2388002C261
:102454000390004FE06006A204B3B34002801990D9
:102464000890E0FEA3E0FF90004FE02FFF50010E24
:10247400900890EEF0A3EFF0A201B34006A202B3DD
:10248400B3500990001AE4F0A3F0802D900890E076
:10249400FEA3E0FF7400D39F74019E401190089046
:1024A400E0F8A3E090001AC8F0A3C8F0800B74FF12
:1024B40090001AF8E4F0E8A3F09000D0E0C394048C
:1024C400400C9008F2E0C3940240030225AD900052
:1024D400B9E0B40147900890E0FEA3E0FF745E12F7
:1024E400779274058E048F05FF127782900890EC22
:1024F400F0A3EDF09000EEE0B4021F900892E0FE2D
:10250400A3E0FF745E12779274058E048F05FF12A8
:102514007782900892ECF0A3EDF08045900890E06B
:10252400FEA3E0FF745E127792740A8E048F05FF97
:10253400127782900890ECF0A3EDF09000EEE0B4F6
:10254400021F900892E0FEA3E0FF745E127792747B
:102554000A8E048F05FF127782900892ECF0A3EDA7
:10256400F0900890E0FEA3E0FF7402BE000CD39F3D
:102574004008752A02752900800A900890E0F52920
:10258400A3E0F52A900892E0FEA3E0FF7402BE00E7
:102594000CD39F4008752E02752D00800A90089276
:1025A400E0F52DA3E0F52E8046900890E0FEA3E030
:1025B400FF7401BE000CD39F4008752A01752900E1
:1025C400800A900890E0F529A3E0F52A900892E0AB
:1025D400FEA3E0FF7401BE000CD39F4008752E01DA
:1025E400752D00800A900892E0F52DA3E0F52E9059
:1025F4000018E529F0A3E52AF0A23BB34009C20183
:1026040090001AE4F0A3F022900053E090038812A3
:1026140077C3E0F542754364900053E0FE9000C434
:10262400E0D39E4037E56075F00884FF7E008F3864
:10263400E56075F00884ADF07C008D3B754008754D
:102644005A03755B96E538C3941F50051211C58073
:102654000690043DE0F5388538438035E56075F033
:102664000884FF7E008F38E56075F00884ADF07C47
:10267400008D3B754008755A03755BB6E538C39405
:102684001F50051211C5800690045DE0F5388538A9
:1026940043229000FAE0F53D754011755A04755BCC
:1026A40000AE52AF53E53D75F00FA4FDACF0EDD391
:1026B4009FEC9E4021E53D8E048F05FF127782ED4D
:1026C40075F010A4FFAEF0E56075F01184FD7C0098
:1026D400ED2FF53E800EE56075F01184FF7E00EF6E
:1026E40024F0F53E853E38E56075F01184AFF07E48
:1026F400008F3B1211C585383FAE52AF539000FA9C
:10270400E075F00FA4FDACF0EDD39FEC9E4028756E
:102714005A04755B10853E381211C5853F398538DA
:102724003AAE52AF53E53D8E048F05FF1277AD8D5F
:102734003B853D3C12123F8538427543642290002C
:10274400FAE0F53D754011755A04755B00AE52AF61
:1027540053E53D75F00FA4FDACF0EDD39FEC9E4026
:1027640021E53D8E048F05FF127782ED75F010A4EC
:10277400FFAEF0E56275F01184FD7C00ED2FF53EAF
:10278400800EE56275F01184FF7E00EF24F0F53EC3
:10279400853E38E56275F01184AFF07E008F3B1200
:1027A40011C585383FAE52AF539000FAE075F00F73
:1027B400A4FDACF0EDD39FEC9E4028755A04755BE4
:1027C40010853E381211C5853F3985383AAE52AF6F
:1027D40053E53D8E048F05FF1277AD8D3B853D3C5F
:1027E40012123F8538427543649000F5E0B40479D1
:1027F400900053E0FE9000C4E0D39E4037E560753E
:10280400F00884FF7E008F38E56075F00884ADF031
:102814007C008D3B754008755A03755B96E538C39B
:10282400941F50051211C5800690043DE0F53885CB
:1028340038438035E56075F00884FF7E008F38E505
:102844006075F00884ADF07C008D3B754008755AC6
:1028540003755BB6E538C3941F50051211C5800695
:1028640090045DE0F5388538432290008EE0B40191
:102874003BE56875F00A84FF7E008F38E56875F0E3
:102884000A84ADF07C008D3B75400A755A05755B72
:1028940012E538C3941150051211C580069005AB9A
:1028A400E0F538E5432538C39464F54390008FE0A0
:1028B400B4013BE56975F00A84FF7E008F38E56951
:1028C40075F00A84ADF07C008D3B75400A755A059D
:1028D400755B7EE538C3941150051211C5800690CE
:1028E4000617E0F538E5432538C39464F543E5421B
:1028F4002543F537900096E0B402109008EAE025ED
:1029040037FE9000EAE0F4042EF5379000EDE0D3B2
:1029140094014040E56CC394E7501D74E7C3956C83
:10292400FE9008ECE08E00F5F0E884FF7E008F381E
:10293400E5372538F537801CE56CC394E7FE90082D
:10294400ECE08E00F5F0E884FF7E008F38E537C3B5
:102954009538F537A2044006E5422464F537E53797
:10296400D394644009E537C39464F537800375371D
:10297400009000C6E0C3953750069000C6E0F537D6
:1029840022D201900076E0A852B800049553503E3C
:10299400900076E0A852B800049553500375370FA1
:1029A400900076E004A852B800049553500375379C
:1029B40007900076E02402A852B800049553500210
:1029C400C201900076E060067409900054F0C233AE
:1029D4007E017F009000CCE01277929000DBE08EC5
:1029E400048F05FF127782E560BC000CD39D40087C
:1029F400D23B740A900054F090008EE0B401099028
:102A040000CDE0C39568400280159000DFE0A85235
:102A1400B8000495535002C201740B900054F09016
:102A2400008EE0B40107E568C394644002801D9001
:102A34000125E0600D900125E0A852B800069553E9
:102A440040028008C201740B900054F0A2014003BC
:102A5400753700C23A90010EE0B4011490010FE002
:102A6400A852B8000495535007E560C3956140022D
:102A7400802A9000B7E0D3941D400B9000B7E0C3C8
:102A8400941EF5378003753700A2374008741590FB
:102A94000054F0D23AD237D235022B7FC235C23736
:102AA400900096E0B40306A22DB3B34003022B7F3B
:102AB4009008EEE0C39405A852B80004955350065C
:102AC4009008F5E06002801F9000B7E0D3941D40A9
:102AD4000B9000B7E0C3941EF5378003753700747C
:102AE4000C900054F0D23A9008EEE0A852B80004DA
:102AF400955350069008F5E07002801F9000B7E0EF
:102B0400D3941D400B9000B7E0C3941EF5378003A7
:102B1400753700740C900054F0D23A9008EEE0A897
:102B240052B80004955350319000D5E0B40228D235
:102B3400339008F4E0FE9008F5E0D39E5006900828
:102B4400F5E0700280099008F4E4F0C23380069046
:102B540008F4E004F08002C2019008EEE02405A825
:102B640052B80004955350139000D5E0B4020A9073
:102B740008F5E07002D2338002C201A232B34027CA
:102B84009000B7E0D3941D400B9000B7E0C3941EAF
:102B9400F5378003753700A2364006741090005450
:102BA400F0D236D23A8002C23685376D9000B7E053
:102BB400D3941D4018900085E02537FE900053E023
:102BC40075F01E84FC7F00EE2CF5378037A23AB3F3
:102BD4004016900085E0FE900053E075F01E84FCE2
:102BE4007F00EE2CF537801C900087E02537FE909F
:102BF4000085E02EFE900053E075F01E84FC7F00FB
:102C0400EE2CF537A23BB34005D233756D0022900C
:102C14000053E075F00584FF7E008F38900053E088
:102C240075F00584ADF07C008D3B754005755A0345
:102C3400755BD69000D9E01475F00584FF7E00E53D
:102C440038BE00039F50051211C5800BE53890046F
:102C54005E1277C3E0F538E5389008EDF09008EDA2
:102C6400E0FE9000C8E0C39E50089000C8E09008C1
:102C7400EDF09000B7E0D3941D401E9008EDE0FE07
:102C8400900085E02EFE900053E075F01E84FC7FDA
:102C940000EE2C9008EDF0803FA23AB3401890006B
:102CA40085E0FE900053E075F01E84FC7F00EE2C5E
:102CB4009008EDF080229008EDE0FE900087E02E71
:102CC400FE900085E02EFE900053E075F01E84FC1B
:102CD4007F00EE2C9008EDF02290008EE0B40136D7
:102CE400E56875F00A84FF7E00900588120048E0CC
:102CF400F547E547D394644010E547C3946475F001
:102D04000F84FF7E008F4780037547009000ABE07F
:102D14002547F54780069000ABE0F54722E5687546
:102D2400F00A84FF7E00900588120048E0C394698D
:102D34004007E568D3946440559000F5E0C39403DC
:102D4400502690088AE0FEA3E0FF7404120039E5DF
:102D540060127792740F8E048F05FF1277829008A9
:102D640088ECF0A3EDF0802490088AE0FEA3E0FF55
:102D74007404120039E562127792740F8E048F0581
:102D8400FF127782900888ECF0A3EDF0800F900892
:102D94008AE0F8A3E0900888C8F0A3C8F0A2044031
:102DA4001A90088AE0FEA3E0FF740312779274017C
:102DB400120039900888EEF0A3EFF090009EE0B482
:102DC4000262E56BC3944175F00584FF7E008F3881
:102DD400E56B75F00584ADF07C008D3B75400575A1
:102DE4005A06755B14E538C3941750051211C58053
:102DF400069006AFE0F538900888E0FEA3E0FF7483
:102E04000A8E048F05FF127782E5388C068D07122F
:102E14007792740A8E048F05FF127782900888ECEB
:102E2400F0A3EDF0900888E0FEA3E0FF90088EE0A8
:102E3400FCA3E0FDEDD39FEC9E400F90088EE0F8DC
:102E4400A3E0900888C8F0A3C8F022E50875F00450
:102E5400A4FFAEF09006CB120048E0903CE8F828BE
:102E64002873804C85537480479000DBE08560F0C4
:102E7400A4FFAEF074081200398F74803385627435
:102E8400802E85687480298569748024856A74809D
:102E94001F856B74801A856C748015856774801027
:102EA400856674800B856D74800690001BE0F57454
:103CE800022E66022E68022E6D022E81022E860298
:103CF8002E8B022E90022E95022E9A022E9F022EB5
:073D0800A4022EA9022EAE59
:102EB400E50875F004A4FFAEF09006CC120048E5D6
:102EC4000875F004A4FFAEF0E0FC9006CD120048B3
:102ED400ECFEE0FFEEC39F4003022FBCE50875F053
:102EE40004A4FFAEF09006CB120048E0B40441E520
:102EF4000875F004A4FFAEF09006CD120048E0C3BC
:102F04009574500AE508F50CD3923C123E4BE50843
:102F140075F004A4FFAEF09006CC120048E0D395FF
:102F240074400AE508F50CC3923C123E4B022FBADA
:102F3400E50875F004A4FFAEF09006CC120048E05A
:102F4400C395745015E50875F004A4FFAEF090061F
:102F5400CD120048E0D395745002800AE508F50CC0
:102F6400D3923C123E4BE50875F004A4FFAEF090FA
:102F740006CC120048E0D395745015E50875F004AA
:102F8400A4FFAEF09006CD120048E0C39574500A39
:102F9400E508F50CC3923C123E4B9006D3E0B40115
:102FA400099000E7E0D395625002800A7402F50CA0
:102FB400C3923C123E4B806AE50875F004A4FFAE50
:102FC400F09006CC120048E0D395744015E50875DE
:102FD400F004A4FFAEF09006CD120048E0C395744F
:102FE4004002800AE508F50CC3923C123E4BE5080A
:102FF40075F004A4FFAEF09006CC120048E0C3952F
:10300400744015E50875F004A4FFAEF09006CD12E7
:103014000048E0D39574400AE508F50CD3923C12BD
:103024003E4B22AE2FAF3074C9BE000CD39F400874
:10303400782F1277E5023141753001752F00AE52B9
:10304400AF53E547BE000DD39F40099000BDE0D3C8
:10305400954840028023754800E547C39553F574AD
:103064009000C0E0D395464008E5462574F54680B7
:10307400069000C0E0F54680020548900099E0D330
:103084009562401CE560C395614015AE52AF53E5AF
:1030940047BE00039F50099000BEE0D3954940020B
:1030A400806E9008EFE0A852B80004955350037561
:1030B4004B009008EFE0A852B8000BD3955340069C
:1030C400E5539008EFF0E54B7041E553C39547F5A0
:1030D40074E574D3940540037574059000BFE0C390
:1030E40095465007E574C3954640028009E546C3FA
:1030F4009574F54680069000BFE0F5469000BFE069
:10310400D3954640069000BFE0F54675490080021D
:103114000549E54B7016900099E0C39562500DE5A2
:10312400472405A852B8000695534002800F90002A
:10313400ACE0F546754B0174789008EFF022AE2FA1
:10314400AF3074E9D39F74039E4008782F1277E55B
:103154000232FB753001752F00754632A22E403DB8
:10316400E54875F00284AFF07E00EF4E70057546B9
:103174001980037546329000ACE075F002A4FFAEEE
:10318400F0E548BE0006D39F4002D22E0548754B99
:103194000374789008EFF0754A000232E2AE52AF41
:1031A40053E5476F4E70030232E2E547BE000DD38C
:1031B4009F40099000BDE0D395484002800F7548B8
:1031C40000E54BC394035003754619800DE547C3CE
:1031D4009553F574E5482574F548900099E0D39526
:1031E40062400E9008EFE0A852B80007D395534010
:1031F40002800C054A9000ACE0B54A03754B00E52B
:103204004BB40306A204B3B34002800A054AE54A5C
:10321400B43C03754B02E54BB402299008EFE0A8D7
:1032240052B8000ED395534009E5539008EFF0755A
:103234004A00900099E0C395625009754A00747879
:103244009008EFF0E54B705A900099E0D3956240F6
:103254001CE560C395614015AE52AF53E547BE000F
:10326400039F50099000BEE0D39549400280087541
:10327400490075464B8028E553C39547F574E574BA
:10328400D394054003757405900099E0D39562408A
:1032940008E5492574F5498006E5492406F549758C
:1032A4004A00E54B7016900099E0C39562500DE515
:1032B400472405A852B80006955340028003754B75
:1032C40001E54BB40118754619054A9000ACE0B508
:1032D4004A06754B02754A0074789008EFF0A20212
:1032E400B34003754632E54675F00AA4FFAEF0908C
:1032F4000894EEF0A3EFF022E570903D0FF8282833
:1033040073023CA8900091E0700302362C9000C731
:10331400E0B4010280030234BF900051E0655F60B5
:1033240009E553455260030234BC7E017F00E5BECB
:10333400127792E5BD2FFF50010E8E5A8F5B9001DC
:103344002CE075F010A4FDACF08C5C8D5DEFD39D8A
:10335400EE9C40091277DD8E5A8F5B8006755B0008
:10336400755A00AE5AAF5B740E1277929000BCE0AF
:103374008E048F05FF127782900898ECF0A3EDF08D
:10338400E56C600FE56CC394FE50089000EDE064BA
:1033940002600280649000DBE0B40B1F900898E0A8
:1033A400FEA3E0FF74E7127792E56C8E048F05FFAD
:1033B400127782900898ECF0A3EDF09000DBE0D354
:1033C400940B40089000C3E064046002802B9008D2
:1033D40098E0FEA3E0FF90089CE0FCA3E0FDEFD39F
:1033E4009DEE9C400D1277DD900898EEF0A3EFF06F
:1033F4008007900898E4F0A3F0900898E0FEA3E01A
:10340400FFEFD39400EE94014008D23B7426900061
:1034140054F0A23BB3B3502C7E057F009000DBE058
:103424008E048F05FF127782900898E0FEA3E0FFD8
:10343400EFC39DEE9C400FAC52AD53740FBC00041F
:10344400D39D50028002C23B900091E0B4022790C9
:10345400089AE0FEA3E0FF900898E0FCA3E0FDEFEB
:103464002DFDEE3CFC74018C068D0712003990088A
:1034740098EEF0A3EFF0900898E0FEA3E0FF900828
:103484009AE0FCA3E0FDEDD39FEC9E4004D2318092
:1034940002B231900898E0F8A3E090089AC8F0A32B
:1034A400C8F09000C3E064016006A231B3B34002E7
:1034B4008006900899E0F56002362AD2317E017FB9
:1034C40000E5BE127792E5BD2FFF50010E8E5A8F94
:1034D4005B90012CE075F010A4FDACF08C5C8D5D6C
:1034E400EFD39DEE9C40091277DD8E5A8F5B8006E8
:1034F400755B00755A00AE5AAF5B740E12779290EA
:1035040000BCE08E048F05FF127782900898ECF0DF
:10351400A3EDF0E56C600FE56CC394FE50089000D9
:10352400EDE06402600280649000DBE0B40B1F9065
:103534000898E0FEA3E0FF74E7127792E56C8E042E
:103544008F05FF127782900898ECF0A3EDF09000BD
:10355400DBE0D3940B40089000C3E0640460028075
:103564002B900898E0FEA3E0FF90089CE0FCA3E009
:10357400FDEFD39DEE9C400D1277DD900898EEF0A0
:10358400A3EFF08007900898E4F0A3F0900898E087
:10359400FEA3E0FFEFD39400EE94014008D23B7405
:1035A40026900054F0A23BB3B3502C7E057F0090CC
:1035B40000DBE08E048F05FF127782900898E0FE0E
:1035C400A3E0FFEFC39DEE9C400FAC52AD53740FCC
:1035D400BC0004D39D50028002C23B900091E0B431
:1035E400022790089AE0FEA3E0FF900898E0FCA36D
:1035F400E0FDEF2DFDEE3CFC74018C068D071200FE
:1036040039900898EEF0A3EFF0900898E0F8A3E062
:1036140090089AC8F0A3C8F09000C3E06401600663
:10362400900899E0F560800375600090008DE0706B
:10363400067570030232FC75BB18023CA8023CA854
:1036440090008DE070030237B57E017F00E5BE1265
:103654007792E5BD2FFF50010E8E5A8F5B9000D3F9
:10366400E0B4010F7E0F7FFFAC5AAD5B1277DD8EA5
:103674005A8F5B9000F8E0B40245AE5AAF5B9000FD
:1036840024E0FCA3E0FDEDD39FEC9E400A900024CF
:10369400E55AF0A3E55BF0AE5AAF5B900026E0FC80
:1036A400A3E0FDEFD39DEE9C400A900026E55AF07E
:1036B400A3E55BF0AE5AAF5B74041200398F6290DD
:1036C40000F8E0704CAE5AAF5B900024E0FCA3E03D
:1036D400FDEFD39DEE9C40091277DD8E5A8F5B80FF
:1036E40006755B00755A00AE5AAF5B741012779280
:1036F4009000F7E08E048F05FF1277828C5A8D5B61
:1037040074FFBC0009D39D4005855B62800375622C
:10371400FE9000C3E0B4010280030237B3A204B3F5
:10372400B3500E900097E0A852B80005D3955350BB
:103734000280719000D4E08562F0A4FFAEF074645E
:103744008E048F05FF1277828C5A8D5BE56C6016B0
:10375400E56CC394FE500F9000EDE0B402089000B5
:10376400DBE0640B60028017AE5AAF5B74E712773C
:1037740092E56C8E048F05FF1277828C5A8D5BAEB6
:103784005AAF5B900898E0FCA3E0FDEDD39FEC9E5C
:103794004005855B60800BA231B34006900899E038
:1037A400F560800BA231B34006900899E0F5608083
:1037B40003756200900090E070067570050232FC9B
:1037C40075BB19023CA8023CA8900090E07003026B
:1037D400389CE55FD3955E400302389A900022E05E
:1037E400FEA3E0FFE5661277D5900022EEF0A3EF8A
:1037F400F09000FDE0B402247E017F00E5BE127764
:1038040092E5BD2FFF50010E8F048E057E0F7FFFC2
:10381400CDCCCD1277DD8E5A8F5B80147E017F0074
:10382400E5BE127792E5BD2FFF50010E8E5A8F5BD5
:103834009000FDE07017AE5AAF5B740A1277927471
:10384400518E048F05FF1277828D668019AE5AAFB0
:103854005B740A1277928F048E057E017F95CDCC1E
:10386400CD1276808F66E566D394644003756664F2
:10387400900022E0FEA3E0FFE5662FFF50010E90CA
:103884000022EEF0A3EFF0900094E0048E048F0584
:10389400FF1277828D6680037566329000E0E070D7
:1038A400067570070232FC75BB13023CA8023CA8E3
:1038B4009000E0E0604A7E017F00E5BE127792E569
:1038C400BD2FFF50010E8E5A8F5B74041200398F86
:1038D400679000E2E08567F0A4FDACF07464FF1229
:1038E40077828D679000E1E08567F0A4FFAEF07405
:1038F400FF8E048F05FF127782ED900075F0800330
:1039040075670090008EE070067570090232FC75D0
:10391400BB17023CA8023CA890008EE0B4010280D0
:10392400030239B07E017F00E5BE127792E5BD2F18
:10393400FF50010E8E5A8F5B9008F0E060199008DA
:10394400F0E01490717212008CE493FC740193FD06
:10395400EDC39FEC9E400280069008F0E014F090C6
:1039640008F0E0C394B3501DAE5AAF5B9008F0E08A
:103974000490717212008CE493FC740193FDEFC304
:103984009DEE9C400280069008F0E004F09008F060
:10399400E0FE9000B4E08E0088F0A4FFAEF0746402
:1039A4008E048F05FF1277828D68800375680090FE
:1039B400008FE0700675700B0232FC75BB16023C7A
:1039C400A8023CA890008FE0B401028003023A5C94
:1039D4007E017F00E5BE127792E5BD2FFF50010EF8
:1039E4008E5A8F5B9008F1E060199008F1E0149012
:1039F40072DC12008CE493FC740193FDEDC39FEC24
:103A04009E400280069008F1E014F09008F1E0C3B3
:103A140094B3501DAE5AAF5B9008F1E0049072DC91
:103A240012008CE493FC740193FDEFC39DEE9C4063
:103A34000280069008F1E004F09008F1E0FE9000A6
:103A4400BAE08E0088F0A4FFAEF074648E048F0593
:103A5400FF1277828D69800375690075BB1F023C74
:103A6400A8023CA87E017F00E5BE127792E5BD2F37
:103A7400FF50010E8E5A8F5B740912779274E68E92
:103A8400048F05FF1277828D6B900096E0700675A7
:103A9400700F0232FC75BB15023CA8023CA89000D2
:103AA40096E07003023BF37E017F00E5BE1277923D
:103AB400E5BD2FFF50010E8E5A8F5B74041200393E
:103AC4008F6A900096E0B401159000EAE0856AF0F0
:103AD400A4FFAEF07407120039EF9008EBF09000E9
:103AE40096E0B402159000EAE0856AF0A4FFAEF017
:103AF4007407120039EF9008EAF0900096E0B403DE
:103B0400028003023BD69000D7E07052E56AC3946A
:103B140019500FD22D9000B6E09008EEF09008F303
:103B2400E4F0E56AD394644004A22D4002802D9011
:103B340008F3E004F09008F3E0FE900129E0B506F4
:103B44000B9008EEE004F09008F3E4F09008EEE047
:103B540064966006900129E07002C22D8063900093
:103B6400B6E070349000EAE0856AF0A4FFAEF07429
:103B7400FF8E048F05FF127782ED9008EEF0AE52AF
:103B8400AF53741EBE0006D39F4002D22DE562D30C
:103B940094E54002C22D8029E56AC3940A500DAE13
:103BA40052AF53741EBE0004D39F50028002D22D24
:103BB400E562D394E54002C22D9000B6E09008EE91
:103BC400F09008EEE0C39405500674059008EEF0FA
:103BD400C232900096E0B40414E56AC3941950020A
:103BE400D232E56AD394324002C232C22D800375C8
:103BF4006A009000EDE070067570110232FC75BB2E
:103C040014023CA8023CA89000EDE07003023C952D
:103C14007E017F00E5BE127792E5BD2FFF50010EB5
:103C24008E5A8F5B90012DE075F010A4FDACF08CE2
:103C34005C8D5DEFD39DEE9C40091277DD8E5A8F2B
:103C44005B8006755B00755A00AE5AAF5B740E124A
:103C540077929000F4E08E048F05FF1277828C5CDB
:103C64008D5D74FFBC00039D5005756CFF8003855A
:103C74005D6CE56C75F00BA4FFAEF09000DBE08E9C
:103C8400048F05FF12778290089CECF0A3EDF0807E
:103C940003756C00900091E0600575BB1A80037594
:043CA400BB188000C9
:103D0F000233050233080236410236440237CA0233
:103D1F0037CD0238B10238B402391902391C0239D1
:103D2F00C50239C8023A65023A68023A9F023AA2BE
:093D3F00023C08023C0B023CA806
:103CA800E57075F00284AFF07E00EF4E7002D2EC42
:033CB80005702272
:0977C3002582F5825002058322A3
:0F008C0025E050020583258250020583F582226C
:10776100EF2F500205832582F582E5833E2EF583B6
:0177710022F5
:1077D500CFC39FFF50011E22C3EF9DFFEE9CFE22EB
:0877E5000806B6000218062296
:0D77A000A3E004F070061277B9E004F022B7
:0E003900048007C3CE13CECF13CFD5E0F6223E
:10768000BC000FBE0008ED8FF084FFADF022E4FED9
:10769000FF22BE000DEF60FE54F0606F20E7030292
:1076A0007736EAC0E0EBC0E078017A0075F001EED1
:1076B00020E710EF25E0FFEE33FE0AC5F023C5F00A
:1076C00030E7F0EA5407F9096A7A007B00600108A4
:1076D000C3EC9E40167004ED9F4010ED9FFDEC9EA4
:1076E000FCE5F0CA4ACA03F5F08005E5F003F5F0C1
:1076F000C3EE13FEEF13FFD9D77908CACBCAD8D08F
:10770000EAFEEBFFD0E0FBD0E0FA22EC8FF084FC45
:10771000ED54F045F0C48FF084FEEDC454F045F014
:10772000C48FF084FDEEC4FE54F02DFFEE540F3CE8
:10773000FEADF07C0022790078008FF0EC7E08200E
:10774000E70DC3CD33CD33C933C9C833C8DEF084A8
:1077500049F9E5F08FF0BE00E6FD7C00E9FFE8FEA8
:017760002206
:0E779200F88FF0A4FFE5F0CE88F0A42EFE22C2
:10000300EF8DF0A4F9A8F0EF8CF0A428F8EE8DF0B2
:06001300A428FEE9FF2213
:10777200600D782B02777C007830D8FED5E0F822B5
:10778200EEC0E07E00127680EFFDEEFCD0E0FE223D
:0C77AD00EEC0E07E00127680D0E0FE22EC
:03001B0002001EC2
:0300530002005652
:03009B00020071EF
:030000000277CCB8
:0977CC0075817675D000024EBDF6
:0B004800E5822FF582E5833EF5832260
:0A77B9000582D58202158315822295
:10001E00C0E0C0F0C083C082C0D075D000124DC009
:0B002E00D0D0D082D083D0F0D0E032E0
:10005600C0E0C0F0C083C082C0D075D000124DC3CE
:10006600D0D0D082D083D0F0D0E032C0E0C0F0C093
:1000760083C082C0D075D000124E21D0D0D082D09D
:0600860083D0F0D0E0324F
:00000001FF
